:03000000020257A2
:060003007F011207ED224F
:03000B00024CF4B0
:10000E00CD30E11520E00FC083C08288828C83CD75
:0C001E00F0D082D08322CDF222CDF62259
:10002A00CB30E11520E00FC083C08289828A83CB5E
:0C003A00F0D082D08322CBF322CBF7223F
:10004600ED30E11320E00EC083C08288828C83E00D
:10005600D082D08322E2226405700EC083C08288DB
:0B006600828C8393D082D08322E6229C
:10007100EB30E11320E00EC083C08289828A83E0E5
:10008100D082D08322E3226405700EC083C08289AE
:0B009100828A8393D082D08322E72272
:10009C0088F0A8817404C0E0C0F018E6C0E008E65F
:1000AC00C0E00886F018188001A3E0C608D5F0F966
:0200BC00F82228
:1000BE00EEC0E0EFC0E088F0E58124FDF8ECC6C0AC
:0900CE00E008EDC6C0E0A8F02234
:0C00D700E0A3FCE0A3FDE0A3FEE0FF229C
:0C00E300ECF0A3EDF0A3EEF0A3EFF02290
:1000EF0075F004AA83AB82D083D082E493A3CAC5F0
:1000FF0083CACBC582CBF0A3CAC583CACBC582CB7B
:08010F00D5F0E8C082C0832294
:10011700E5F06010C3EC13FCED13FDEE13FEEF13D7
:05012700FFD5F0F022FD
:10012C00120235C380021819E637F6DAF9020226F4
:10013C00E0A3FEE0FFEF8DF0A4CFC5F0CCA42CFC27
:09014C00EE60038DF0A42CFE22EC
:10015500C2D1C2D5EE30E707D2D1D2D5120202EC18
:1001650030E705B2D112020A12017D30D103120225
:100175000230D50312020A22BC000EBE0032EF8DFA
:10018500F08420D226FFADF0227B0075F008EF2F1A
:10019500FFEE33FEEB33FBEE9DEB9C4005FBEE9D46
:1001A500FE0FD5F0E9E4CECDCBCC227EFF7FFF223A
:1001B500EDB410005022EE8DF084FEEF54F045F0C2
:1001C500C48DF084C4FCEF540FC445F0C48DF08495
:1001D500FFADF0E4CC4FFF22EE8DF08420D2CC7E33
:1001E50008CEC5F0CDCBEF2FFFED33FD10D7079B24
:1001F5005005D5F0F1229BFD0FD5F0EA22C3E49F0F
:0D020500FFE49EFE22C3E49DFDE49CFC226C
:0C021200EE30E707E4C39FFFE49EFE22ED
:10021E0074F9800674FA800274FCD083D082258132
:07022E00F581C082C08322AC
:0F023500E5D054182407F8E58124FCF97A042257
:10024400EFB40A077F0D1202447F0A3099FDC29968
:030254008F99225D
:0F02570075813BE4787FF6D8FD75A0FF02509FBC
:08026600C2047524011200031B
:10026E001249B98F25E52514600B146019146036F8
:05027E00146043804400
:10028300E524B40101D34004152480387524068085
:0602930033E524B4060669
:06029900120003E4FF2245
:10029F00AF24121DDA8F26E526B404037F04223023
:1002AF000416E4FF22E524B4060050040524800858
:1002BF0075240180037F0422E524B4040302041E85
:1002CF005014E52414602114700302037614700394
:1002DF000203D90205FEE52424FB70030204631414
:0802EF0070030204D002026E4C
:1002F7007B027A0079007D057C15786912081D7FDD
:10030700017B027A007900124907900106E0700B21
:100317007F027B057A15797A124907900106E0FA80
:10032700B4010B7F027B057A15798B12490790017F
:1003370006E0FAB4020B7F027B057A15799C124915
:1003470007900106E0FAB4030B7F027B057A157963
:10035700AD124907900106E0FAB4040280030205D2
:10036700FE7F027B057A1579BE12490702026E7B72
:10037700027A0079007D057C1578CF12081D7F0170
:100387007B027A0079001249079000FDE060079030
:10039700010CE0B401117B027A0079007D057C1520
:1003A70078E012081D801D9000FDE0FDE4C0E0C06C
:1003B700057B027A0079007D057C1578F112081D0E
:1003C700158115817F027B027A00790012490702A5
:1003D700026E7B027A0079007D057C16780312088D
:1003E7001D7F017B027A0079001249079000FBE02C
:1003F700C0E0A3E0C0E07B027A0079007D057C16AF
:10040700781412081D158115817F027B027A007905
:100417000012490702026E7B027A0079007D057C93
:1004270016782412081D7F017B027A007900124991
:1004370007900102E0C0E0A3E0C0E07B027A007908
:10044700007D057C16783512081D158115817F0200
:100457007B027A00790012490702026E900106E0DA
:0E046700FA64026009EA64036004EAB4041651
:10047500E525B401021524E525B403028003020530
:10048500FE052402026E7B027A0079007D057C164A
:10049500784512081D7F017B027A00790012490711
:1004A500900104E0C0E0A3E0C0E07B027A0079009F
:1004B5007D057C16783512081D158115817F027B17
:1004C500027A00790012490702026E7B027A0079EE
:1004D500007D057C16785612081D7F017B027A0087
:1004E5007900124907900106E0601514603E14601A
:1004F500671470030205881470030205B30205DC56
:100505009000FBE0C0E0A3E0C0E09000FDE0FDE46A
:10051500C0E0C0057B027A0079007D057C1678670E
:1005250012081D74FC2581F5810205DC9000FBE0B5
:10053500C0E0A3E0C0E09000FDE0FDE4C0E0C00540
:100545007B027A0079007D057C16787812081D7487
:10055500FC2581F5810205DC9000FBE0C0E0A3E00D
:10056500C0E09000FDE0FDE4C0E0C0057B027A003C
:1005750079007D057C16788912081D74FC2581F5A6
:100585008180549000FBE0C0E0A3E0C0E09000FD56
:10059500E0FDE4C0E0C0057B027A0079007D057CC2
:1005A50016789B12081D74FC2581F5818029900021
:1005B500FBE0C0E0A3E0C0E09000FDE0FDE4C0E0AA
:1005C500C0057B027A0079007D057C1678AD12089E
:1005D5001D74FC2581F5819000FDE0600790010CFC
:0405E500E0B4010A73
:1005E9007420900005F07441A3F07F027B027A0029
:0805F900790012490702026EAD
:0606010075240112000344
:100607001249B98F25E52514600F14601D14607613
:0906170014700302069D0206A006
:10062000E524B40101D340041524807475240580A9
:060630006FE524B405068D
:06063600120003E4FF22A4
:07063C00900115E0B4011567
:10064300AF241224728F26E526B404037F042230DC
:050653000436E4FF2263
:100658001200037F017B057A1979C91249077F02C5
:100668007B057A1979DA1249071249A6E4FE7FFA5E
:1006780012498E1249A67E077FD012498E120003B6
:10068800E4FF228013E524B4050050040524800803
:1006980075240180037F0422E52414600E14601C75
:0B06A80014602A146038146046805370
:1006B3007B027A00795E7D057C1978EB12081D8038
:1006C300427B027A00795E7D057C1978FC12081D55
:1006D30080317B027A00795E7D057C1A780D1208E1
:1006E3001D80207B027A00795E7D057C1A781E12BC
:1006F300081D800F7B027A00795E7D057C1A782FB6
:1007030012081D740690005EF07F017B027A007967
:100713005E1249077B027A00795E7D057C1A784078
:1007230012081D7405900062F004A3F07F027B029F
:0A0733007A00795E124907020607FA
:10073D002053746172742043686172676572202062
:10074D0000202020202020202020202020202532A5
:10075D00642000205374617274204469736368616E
:04076D00726765004A
:050771008F2475250036
:10077600E52424FD601214601E24FE600514600E3C
:02078600801ED3
:100788007F06124C15227F07124C152220970F7FE7
:1007980006124C15222096067F07124C15220525B5
:0907A800E525B464C9E4FEFF225A
:0307B100752400AC
:1007B4002097067F05124C15220524E524B464F025
:0407C400E4FEFF222E
:0A07C80075D90275E90075F90022E9
:0B07D200EEB40005EFB40001D34007B7
:0807DD00EF1F70F11E80EE22F7
:0807E5008F3AD28212482B2248
:0807ED008F3AC28212482B2250
:0907F500C2A3C2A2D2A1D2A0222B
:10080000A881058118EBC6C908CAC6CA08F67BFFCD
:10081000112ED0E0D0E0D0E0C082C08322D083D0BF
:1008200082EDC0E0ECC0E0E8C0E0C082C083E581BA
:10083000F82425F58108E8C9CBF709EAF709EBF7B1
:1008400009770009E924F6FA75F000C2D5E924FC1D
:10085000F8E924F9F9ECC0E0E8C0E0D1E51200467F
:10086000FFE92409F9D0E0F8D0E0FCEF605020D592
:1008700074B4250AE4FB74FFFCF7D2D580D3D1FE13
:1008800080CFFF20F71CBCFF067014D2F380C2ECAF
:10089000C0F075F00AA42FD0F030F703F78001FC08
:1008A00080AFB7FF03EF80F4E780E57F00D1FE194A
:1008B0001709800DEF24D0B40A0040C68093B6FF1C
:1008C000EAE581C39421F581E4FED0E0FFD082D037
:1008D00083D0E004600ED083D0821581158115810C
:1008E000C082C08322900F78E49360256FA36006D6
:1008F000A350F5A380F293FF400442F080BEE4A32E
:10090000938F83F582E4C2D130F705B7FF027700F9
:100910007340A1D3A380D1EAC8FDE620F703FC8091
:1009200001F71A1AEDF88094D2D17F7880027F58AF
:10093000D17990100421CCBCFF05B7FF02805AC0CA
:10094000F08AF0EAC92420F583E8FEECC0E0D1E5A6
:10095000120046FF601AC583C9C583F70B19E9C5A4
:1009600083F908B800010CEE2404F9E7C39B70E09A
:10097000D0E0FCE5F024FDFAD0F08B82A98309EEEB
:10098000C394FBF583F805828004E7F60809D58255
:10099000F9A9831819C2F0414F8AF0EAC9F583E832
:1009A000FED1E5120046FF6013EEC8CE8D82D1FE67
:1009B000AD82EEC8CE08B800EA0C80E7A983E5F066
:1009C00024FDFA01487F30D179900806C2F7D18919
:1009D000E8CAC9C88049D2F7EA147D0230F4047D20
:1009E0000424FEF8E68A83A88330E70DD2D1C3E45D
:1009F00096F618DDFAA8838000C2F7D179900A052F
:100A0000D189C9C8CAC9B1FF8015D179E618188043
:100A100004D1797425C2F7F70BCAC9C8CAC2F0E776
:100A2000FDE924002BF8B6300318DBFABB00080BF5
:100A300008BD00031B8013BDFF02800EEDC39BFEAB
:100A40004008600674305192EDFBEB70020148ECF7
:100A5000046023D39B401F601DFE7D2020F13830B1
:100A6000F3027D3030F023BD3018518E18EF30E6A0
:100A700001187111804030F03F71110B30F6390BC5
:100A80008036EF71111E30F6011E518E8028EE6007
:100A900005ED08F6DEFC2230F00771110B30F6018F
:100AA0000BE9FF2420F9E6F71918DBFAEDF719DE58
:100AB000FCEFF92420F8CCCBEB700201481919E8BF
:100AC000C0E0E6FFD1E50909EFD16AD0E0F818DB14
:100AD000EE090901481A1AD181900F6CE6086002EC
:100AE0002406936023F7190B30E504E4A380F3EBAD
:100AF000C0E0743AF7E924FCF908901004D1891891
:100B0000D0E02405FBE92404C8CAC9E92420F88000
:100B1000AC08EFF68FF030F604743008F622619BD3
:100B2000C2F79159BFFF0261ADEF60F22481FF204F
:100B3000E73618040FD113EBC39F60124010FDFE7F
:100B40000BE89FF8742EC618C6DDFC18805DF4040F
:100B5000FD7E000DE824F9F880057430F6180BDDF1
:100B6000F9742EF60B188043F4FD7E070DBD0700C7
:100B70004016E9FD097430F709E9C39870F7EDF9FB
:100B800080087430F60E0B08DDF8742EF6080B0B97
:100B90007430F6D113E8C39BF88010E92420F87470
:100BA00030F618742EF6187B027E00B1AD414AC2B1
:100BB000F78002D2F79159BFFF0280F1BF000E7497
:100BC00030F618742EF6087E007B02800EEF24812A
:100BD000FF18742EC608C6EBFE1E0BD113E8C39B8C
:100BE000F8EFC0E0B1ADD113D0E0FFC0F0E8C39B97
:0E0BF000F8E730F704746580027445F618EFDC
:100BFE0020E704762B8004762DF4041875F00A8411
:100C0E002430F618E5F02430F6EB2404FBD0F0D1B6
:100C1E002918B1FF61ADC2F78002D2F7D2F2915915
:100C2E00BFFF0261ADE7B4FF037406F7BF7B004060
:100C3E0016EF248120E706C397600C500A74822FAA
:100C4E00C7C397F7020B2917020BBCD179ECC0E092
:100C5E00C0F018E63308E63392D5186033B4FF407F
:100C6E00E6C2E76009900FBCC2D17B078007900FE8
:100C7E00C3D2D17B06E493F709A3DBF97B0330D112
:100C8E000A742B30D502742DF70B09197C80A184C0
:100C9E00EAC0E074307A08F709DAFC097C81A17D9C
:100CAE00CAC0E0EA75F010A4CAABF075F04DA42BE3
:100CBE00FBE435F0FCEA2410FAEB34C5FBEC34D936
:100CCE00FCE6C2E7FF75F056A4F42411C5F0F43427
:100CDE00C58FF0A42AE5F03BE43CFBC0E0E9C0E0A0
:100CEE00E8C0E0EBC0E020E707800812112C801F5F
:100CFE00F404FB121411D0F0D0E0F8C0E0187583A4
:100D0E000418E6C0E008D583F930F7DF121288D058
:100D1E00E0F8D0E02408F9EED2E7CE33EF332482A8
:100D2E00FAECFBD0E0FCE4C3CB33CBCD33CDCE33EA
:100D3E00CE33DAF37A0875F00A8460062430F71998
:100D4E001A0CE5F02430F7198BF0740AA4FBAFF0FF
:100D5E008DF0740AA42FFDAFF050010F8EF0740ABF
:100D6E00A42FFE743035F0F719DADDE9240AF9D034
:100D7E00E0FAE9D39AFBECFF247FFFCAC9C824FD31
:100D8E00FAE9FD09EF046003120F2FEDF909EF04E4
:100D9E006003120F2FEDF9D0F0D0E0FC7B0722E7B5
:100DAE00B4FF027406700820F0010E8E838016C305
:100DBE009E400EF583603674300BF618D583FA809C
:100DCE002CF404F583C0E0E9C0E0E8C0E0F92B04A0
:100DDE00F8EEC0E0EFC0E009120F2DD583FAD0E097
:100DEE00FFD0E0FED0E0F8D0E0F9D0E0FD08D12948
:100DFE0018D2F07F2D20D10C7F2B20F5077F2020DD
:100E0E00F602C2F0228982E92420F98B83E6F719D3
:100E1E0018D583F9A982E92420F822E9F582240164
:100E2E00F98B8330F22A20F027C2F2E608B42E02A4
:100E3E00D2F2D583F6E8C39BF88B8330F210E6B47A
:100E4E003005081BD583F7B42E07081B8006D2F297
:100E5E00E6F70908D583F9E9F8A98222BDFF051244
:100E6E000244800312000E09071922E9CAC8E924B8
:100E7E0001F922E9CAC8E92420F922A2F492D5C0C8
:100E8E00F0E582FD30D50623F582FD181818E685AB
:100E9E0083F084F620D5047B0180027B0308E5F005
:100EAE00D6C6C48583F084C4C6C445F0C48583F019
:100EBE0084D6DBE9E5F024F6500730D10224202455
:100ECE0007243AF70920D509DDC3D0F01818AB82F4
:100EDE0022DDB8181880F3E7F819E7FC19E7FDBD15
:100EEE00FF0122090907B70004190719221919224F
:100EFE00CACDE8C0E0E9C0E0E6FB08E6FA08E6F98C
:100F0E00EFBBFF05120244800A06B600031806085E
:100F1E0012002A080618D0E0F9D0E0F8CDCA22E96E
:100F2E00FD1BE7B4350FEBFE600709E719F709DE85
:100F3E00F718EDF92240EF09C3E899601AE719B4E2
:100F4E002E04F70980F104B43A067430F70980E7ED
:100F5E00F709E899FE80D1197431F70B80D4286E09
:100F6E00756C6C290049584450434C046C10620057
:100F7E00680023012D022B2020402E80002A091705
:100F8E006F09C578092858092E7309377509F96450
:100F9E0009D66909D6630A0A250A11700AD5660BA5
:100FAE0020650BB3450BAF670C28470C240020209F
:0B0FBE0020204E614E202020464E49AE
:100FC9001200D7EFB2E7FF80031200D7E58124FDB5
:100FD900F8F9E63308E63370060213B60213A504DE
:100FE90060FAEE33EF33700EE6FF18E6FE18E6FD01
:100FF90018E6FC0213B60460E3E58124FBF8D3ECA0
:101009009608ED9608EE9608EFC2E786F0C2F795C6
:10101900F0400FEFC6FF18EEC6FE18EDC6FD18EC3E
:10102900C6FC1213C7C3EB9FF5F0700EE58124FBD4
:10103900F9E4C3CC20D5730211049418605C400E06
:10104900E4FF19E7FE19E7FD19E7FC0210E0E4FFE8
:1010590030F405CEFCE4CDFF30F305E4CECDCCCFA2
:1010690030F21AE5D054184404F8EF54F0D6C4FF0E
:1010790008ECD6C4FC08EDD6C4FDEEC4FE740355D5
:10108900F06012F5F0C3EE13FEED13FDEC13FCEF67
:1010990013FFD5F0F030D55D8009E4CEFFE4FDFC07
:1010A90030D552C3E49FCC191919C797CD09C797F1
:1010B900CE09C797FF4E4D4C70140213B6DB0302DD
:1010C90013A9EC2CFCED33FDEE33FEEF33FFEF30CB
:1010D900E7EBECCFCECDFCEF30E70D0CBC00090DF2
:1010E900BD00050EBE00010BEB7005A2D102139DD8
:1010F900A2D10213B0E42FCC19191937CD0937CE73
:101109000937FF50090BEB700CA2D102139DEFCEEA
:10111900CDCCFF80C2EF13CE13CD13CC13FF80B714
:101129001200D7EF4E601AE58124FEF924FEF8E794
:1011390019477019EE33EF33B4FF030213A50213F5
:10114900A9E58124FDF8E63308E63380EB1213C7DD
:10115900248150082B5008A2D502139D2B50DFF78C
:10116900FAE61846197020B7800DEE33CAA2D513D6
:10117900FFCA13FE0213B6EC4D703CBE8046E6FC76
:1011890008E6FD08E680E4EC4D7039BE800280EE89
:10119900E4CEC7CDC6F5F008E4C6CCF9FBFFFA806A
:1011A90076E4CEC9E4CDCAE4FFCCFB803CE4C9CDEA
:1011B900CFCBECCACC8060E4F9FAFBFFCECDCCC52D
:1011C900F00880538CF0E660D8A4C5F0CDFAC5F0DC
:1011D900E6A42DCEF9C5F03400FDE6A42DC5F03402
:1011E90000FDCCFBC5F0CC7F0008E660C0A42EC58D
:1011F900F03C50010DCAFCC5F0CEE6A42AC5F03D6D
:1012090050010FC9FDC5F0CAE6A429C5F03F79010F
:10121900400119CBC5F0CF08E6A42AC5F03F500517
:101229000BBB000109CCC5F0FAE6A42CC5F03B5074
:101239000109CDC5F0CCE6A42DFDC5F039FE330872
:10124900500906B60011A2D502139DEA33FAEC3310
:10125900FCED33FDEE33FEEA30E7140CBC00100D53
:10126900BD000C0EBE000806B60004A2D580D9E662
:05127900A2D50213B034
:10127E00D083D0820213A91200D7EFC2E74E7003BB
:10128E000213A5C082C083E58124FBF8F9E6084667
:10129E0060DE1213C70FBF0006D083D08280E1EF4D
:1012AE0024805007C3CB9B500D80C5CB9B4007D0ED
:1012BE0083D08202139DF6F583EC4D701FBE801C09
:1012CE00E58124FBF8E583A2D513FFE692E7FE182D
:1012DE00E6FD18E6FCD083D0820213B6E58124FB2E
:1012EE00F8E6CEF618E6CDF618E6CCF6EFCCFFE82B
:1012FE002402F9F8E7FA19E7FB19E7FCE4F5F075B3
:10130E00821A758380801DE58303F58330E706A777
:10131E00F009E4F5F0C3EF33FFED33FDEE33FE409D
:10132E000C30E717C3EF9CED9BEE9A400EC3EF9C7B
:10133E00FFED9BFDEE9AFEE58342F0D582C9E7FAFA
:10134E0019E9F81919E720E7191ABA000302127EF3
:10135E00E5F025F0FFE633FC18E633FD18E633FE24
:10136E008009FE09E7FDE6FCE5F0FFEF30E7160C1D
:10137E00BC00120DBD000E0EBE000A0A7007D0830F
:0F138E00D08202139DEAA2D5D083D0820213B081
:10139D0074FF13FF7E80800774FF8001E4FFFEFD64
:1013AD00FC800613FFEE92E7FED0E0F8D0F0E58169
:1013BD0024FCF581C0F0E8C0E022E7D2E7C733098D
:1013CD00E733FB92D592D1EED2E7CE33EF33FF5018
:0413DD0002B2D52261
:1013E1003F8000003DCCCCCD3C23D70A3A83126F1D
:1013F10038D1B7173727C5AC358637BD33D6BF953A
:10140100322BCC7724E69595179ABE150A4FB11F5A
:10141100EB60105407700AEB543803241C12143C7F
:1014210022232312143CEB543870012203241CFBA9
:101431001200BEEB12143C12112C229013E1FC930A
:0E144100FF0CEC93FE0CEC93FD0CEC93FC22E4
:10144F001214958000EC3392D550031214837A2036
:10145F00C3EC20E712EF33FFEE33FEED33FDEC3339
:10146F00FC20E703DAEF22EA247DA2D513FFEC92EA
:10147F00E7CEFC22E4C39FFFE49EFEE49DFDE49CC7
:10148F00FC22C2D580C8EED2E7CE33EF3392D524FB
:10149F0081400CE4C2D5A2D513FC33FDFEFF2224FC
:1014AF00E0500474FF80EFF404FAE4CCCDCECF808B
:1014BF000DC3EF13FFEE13FEED13FDEC13FCDAF18A
:1014CF0020D507EECDFEEFCCFF22E4C39CFCE49DBC
:1014DF00FDE49EFEE49FCCFFEECDFE22EFC2E7FFC0
:1014EF0080A47A083392D5E4FDFEFF30D5031214A1
:1014FF0084EC334010EF33FFEE33FEED33FDEC336E
:10150F00FCDAEE80BEEA247EA2D513CC92E7CDCED4
:03151F00FF80B09A
:10152200E58124FEF88FF063F080E6F96480B5F07F
:101532001B188EF0E6B5F014188DF0E6B5F00D1814
:101542008CF0E6B5F006E4FFFE0213B68FF030F73A
:101552000689F030F701B340077F017E000213B61F
:0715620074FFFFFE0213B647
:101569004241545445525920545950452020202075
:10157900003A4E69434420202020202020202020AA
:1015890020003A4E694D482020202020202020208C
:101599002020003A4C69506F202020202020202054
:1015A900202020003A4C69494F4E2020202020203D
:1015B90020202020003A534C4120202020202020A8
:1015C90020202020200042415454455259204345AF
:1015D9004C4C20202020003A4155544F204445547A
:1015E90045435420202020003A2532642020202021
:1015F90020202020202020202000424154542E2049
:1016090043415041434954592020003A2534646DDF
:1016190041682020202020202020004348415247B3
:10162900452043555252454E542020003A253464F2
:101639006D412020202020202020200044495343B0
:10164900482E2043555252454E54202000455849B2
:1016590054204241545445525920202020004E69BB
:1016690043442025326443202534646D4168004E8B
:10167900694D482025326443202534646D41680052
:101689004C69506F202025316443202534646D4115
:1016990068004C69494F4E20253164432025346444
:1016A9006D416800534C4120202025316443202599
:1016B90034646D41680053455420424154544552A5
:1016C90059205459504500204E6943442020202078
:1016D9002020202020202000204E694D4820202055
:1016E900202020202020202000204C69506F20201D
:1016F90020202020202020202000204C69494F4E06
:10170900202020202020202020200020534C412070
:101719002020202020202020202020005345542054
:10172900424154544552592043454C4C00202532DE
:101739006420202020202020202020202020005349
:101749004554204341504143495459202020200009
:10175900202534646D41682020202020202020008D
:10176900202534646D4120202020202020202000C5
:101779004C4F41442046524F4D204C4F432E253269
:1017890064005341564520544F204C4F432E20208E
:10179900253264004552415345204441544120417A
:1017A9005420253264004C6F6164696E6720426180
:1017B9007474657279200046726F6D204C6F636195
:1017C90074696F6E2025326400204E6F2042617467
:1017D90074657279204461746100204174204C6FF2
:1017E900636174696F6E2025326420004F5645523B
:1017F900575249544520444154413F2000205361E8
:1018090076696E672042617474657279200020548C
:101819006F204C6F636174696F6E202532642000FC
:10182900455241534520444154413F202020202026
:101839000045726173696E672042617474657279DB
:1018490020002045584954204D454D4F52592020DC
:10185900202000204E69434420253264432025344A
:10186900646D416800204E694D482025326443204B
:101879002534646D416800204C69506F2020253162
:101889006443202534646D416800204C69494F4EFA
:101899002025316443202534646D41680020534C70
:1018A9004120202025316443202534646D4168009E
:1018B90020454D5054592020202020202020202030
:1018C900002020202020202020202020202020202F
:1018D9002000455241534520414C4C20444154413C
:1018E9003F200045726173696E6720416C6C20442A
:1018F9006174610020202046726F6D204D656D6F07
:1019090072792020005345542043454C4C532044C0
:10191900455445435400204155544F202020202050
:1019290020202020202000204D414E55414C2020D0
:101939002020202020202000534554204348415294
:10194900474552204D4F444500204359434C4520BB
:1019590043484152474520202000204348415247EF
:0B19690045204F4E4C5920202020004C
:1019740020444953434841524745204F4E4C592037
:101984000053455420434841524745204359434C52
:10199400450053455420534F554E4420564F4C5503
:1019A4004D4500204F4E20202020202020202020A4
:1019B40020202000204F46462020202020202020C8
:1019C400202020200020202A2A204552524F522035
:1019D4002A2A2020200020204D656D6F7279204630
:1019E40061696C20202000204C4F4144202020209D
:1019F40020534156452020002053415645202020A5
:101A04002020455241534520002045524153452052
:101A1400202020464F524D41540020464F524D4104
:101A2400542020204558495420200020455849542A
:101A340020202020204C4F41442020005573652055
:101A44003C3E20746F2053656C65637400204E6FB8
:101A540074204170706C696361626C652000466F2C
:101A6400722054686973204261747465727900202D
:101A7400466F722054686973204D6F64652020009E
:101A84002043454C4C5320444554454354494F4E00
:101A9400003A4155544F202020202020202020208F
:101AA40020003A4D414E55414C202020202020203A
:101AB4002020002043484152474552204D4F444581
:101AC400202020003A4359434C4520434841524783
:101AD40045202020003A434841524745204F4E4C70
:101AE4005920202020003A44495343484152474555
:101AF400204F4E4C59200020434841524745204333
:101B040059434C45202020003A4E6F742041707098
:101B14006C696361626C65200020534F554E44200C
:101B2400564F4C554D45202020003A4F4E20202042
:101B340020202020202020202020003A4F4646202C
:101B4400202020202020202020202000204558492B
:101B540054204F5054494F4E5320202000204241DE
:101B6400545445525920204D454D4F525900204D53
:101B7400454D4F525920204F5054494F4E53002049
:101B84004F5054494F4E532020202045584954006B
:101B9400204558495420202020424154544552594C
:101BA400002020534D41525420434841524745524E
:101BB4002000202053455256494345204D4F44456B
:101BC40020200020204649524D5741524520312EB5
:101BD400313220002020202852454C4541534520D5
:101BE400332920200020444953434820432D535493
:101BF4004550202020003A25346420202020202035
:101C04002020202020002043555252454E5420537A
:101C14005445502020200020535441525420444520
:101C24004C415920202020003A2533642053656319
:101C34006F6E647320202020002044495343482DB4
:101C44004348472044454C415900204D41582E20DB
:101C5400564F4C542F43454C4C20003A25352E32D8
:101C640066562020202020202020202000204D49BE
:101C74004E2E20564F4C542F43454C4C2000204EA2
:101C84006943442053454E53495449564520003A2C
:101C9400253264206D562F43656C6C202020202053
:101CA4002000204E694D482053454E53495449560F
:101CB40045200020535550504C59204D4F4E495407
:101CC4004F5220003A4348253164202020202535F6
:101CD4002E32665673200020564F4C5441474520FF
:101CE40053544550202020003A25346420202020DD
:101CF40025352E3266562000204558495420534538
:101D0400525649434520202000534554204449530A
:101D1400434820432D5354455000534554204355C4
:101D24005252454E54205354455000534554205369
:101D3400544152542044454C4159200053455420A9
:101D440044495343482D4348415247450053455461
:101D5400204D41582E20562F43454C4C20003A2507
:0F1D6400352E32665620202020202020202000FF
:101D7300534554204D494E2E20562F43454C4C205D
:101D8300004E6943442053454E5349544956452018
:101D930020003A2532646D56202020202020202068
:101DA300202020004E694D482053454E5349544945
:101DB300564520200053455420535550504C59202C
:101DC3004D4F4E2E200053455420564F4C544147FF
:071DD3004520535445500068
:051DDA008F2712000339
:101DDF00900106E0601214600F14606C14606914B7
:081DEF007003021E7A021E9B24
:101DF7009001077405F0A37478F07401900116F050
:101E070075280A75290F752AA09000FDE0FBE433B9
:101E1700E4500114FCFD7E00AF03121454C004C04B
:101E270005C006C007E4FCFD7496FE7444FF12115A
:101E37002CC004C005C006C0077CCD7DCC7E4C7F7E
:101E47003E12112C1214958E2B8F2C752D01804468
:101E57009001077410F0A37468F07402900116F0F3
:101E670075280375290F752AA0E4F52BF52C752D18
:101E77000180219001077409F0A374C4F0740290E3
:101E87000116F075280675291B752A58E4F52BF5F8
:101E97002C752D031249B98F2EE52EB40403AF2EEE
:101EA70022E52714601B14700302215114700302EA
:101EB70021C11470030223081470030223CA021DF0
:011EC700DF3B
:101EC8007F017B057A1679BF124907E52EB4011503
:101ED800900106E0B40001D34005E014F0800674D8
:0F1EE80004900106F0E52EB4020280030220B53B
:101EF7009000FBE0FAA3E0FB900102EAF0A3EBF00D
:101F0700900102E0B40005A3E0B464005009900119
:101F170002E4F0A37464F0900102E0FEA3E0FFE4A2
:101F2700FC7D6412017DEE900102F0A3EFF09001B9
:101F370002E0FEA3E0FFE4FC7D64120141EE9001A4
:101F470002F0A3EFF0BE0B04BFB801D3400A900123
:101F570002740BF0A374B8F09000FBE0FAA3E0FB67
:101F6700EAB52905EBB52A01D3400A9000FBE5291C
:101F7700F0A3E52AF07F05124C158E2F8F30E4FC75
:101F8700FD90011CE0FEA3E0FF121491C004C00500
:101F9700C006C00774CDFC14FDFE743DFF12112C62
:101FA7008C318D328E338F34E4FCFDAE2FAF30127F
:101FB7001491C004C005C006C007AC31AD32AE33C2
:101FC700AF34121288C004C005C006C0077466FE8D
:101FD700FCFD743FFF121522BF010280030220A9F6
:101FE700900106E0600F14600C1460431460401405
:051FF70060770220AF3D
:101FFC00E4FCFDAE2FAF30121491C004C005C00636
:10200C00C007AC31AD32AE33AF34121288C004C04D
:10201C0005C006C0077455FEFCFD743FFF12112C61
:10202C00121495EF9000FDF08079E4FCFDAE2FAF1B
:10203C0030121491C004C005C006C007AC31AD32DB
:10204C00AE33AF34121288C004C005C006C0077C82
:10205C00DD7D607E8A7F3E12112C121495EF90006C
:10206C00FDF0803FE4FCFDAE2FAF30121491C004A4
:10207C00C005C006C007AC31AD32AE33AF3412125E
:10208C0088C004C005C006C007E4FEFCFD743FFF19
:0D209C0012112C121495EF9000FDF080063B
:1020A900E52D9000FDF01249A6E4FF22E52EB403C8
:0120B9001313
:1020BA00900106E0B404005005E004F08005E490C5
:1020CA000106F0900106E0700F7B027A0079147D18
:1020DA00057C1678D012081D900106E0FAB4010FAB
:1020EA007B027A0079147D057C1678E112081D902E
:1020FA000106E0FAB4020F7B027A0079147D057CAE
:10210A001678F212081D900106E0FAB4030F7B025A
:10211A007A0079147D057C17780312081D90010650
:10212A00E0B4040F7B027A0079147D057C177814D9
:10213A0012081D7406900014F07F027B027A00795F
:10214A0014124907021DDF7F017B057A17792512D0
:10215A004907E52EB401109000FDE0B52D01D340EA
:0C216A00069000FDE014F0E52EB4020623
:102176001249A6E4FF22E52EB4030F9000FDE0B558
:10218600280050069000FDE004F09000FDE0FBE41E
:10219600C0E0C0037B027A0079147D057C1778368F
:1021A60012081D158115817406900014F07F027BBC
:1021B600027A007914124907021DDF7F017B057A36
:1021C6001779481249079000FBE0FAA3E0BA00032A
:1021D600B4640050099000FBE4F0A37464F090002E
:1021E600FBE0FAA3E0FBEAB52905EBB52A01D340EB
:1021F6000A9000FBE529F0A3E52AF0E52EB40120BC
:102206009000FBE0B40006A3E0B46401D340119053
:1022160000FCE024CEFB9000FBE034FFF0A3EBF0E3
:0A222600E52EB4020280030222B389
:102230009000FBE0FAA3E0FB900102EAF0A3EBF0D0
:10224000900102E0B40005A3E0B4640050099001DD
:1022500002E4F0A37464F0E4FCFD900102E0FEA34C
:10226000E0FF121491C004C005C006C0077C0A7DBF
:10227000D77E237F3C12112C121495EE900102F0B0
:10228000A3EFF0900102E0FEA3E0FFE4FC7D641206
:102290000141EE900102F0A3EFF0BE0B04BFB801C4
:1022A000D3400A900102740BF0A374B8F01249A64F
:1022B000E4FF22E52EB4031F9000FBE0B52905A33F
:1022C000E0B52A0050119000FCE02432FB9000FBA6
:1022D000E03400F0A3EBF09000FBE0C0E0A3E0C02E
:1022E000E07B027A0079147D057C17785912081D6D
:1022F000158115817406900014F07F027B027A002C
:102300007914124907021DDF7F017B057A167924B3
:10231000124907900102E0FAA3E0BA0003B4640096
:102320005009900102E4F0A37464F0900102E0FA15
:10233000A3E0BA0B04B4B801D3400A900102740BB5
:10234000F0A374B8F0E52EB40120900102E0B400CF
:1023500006A3E0B46401D34011900103E0249CFB88
:0F236000900102E034FFF0A3EBF0E52EB402068B
:10236F001249A6E4FF22E52EB4031F900102E0B448
:10237F000B05A3E0B4B8005011900103E02464FBF7
:10238F00900102E03400F0A3EBF0900102E0C0E016
:10239F00A3E0C0E07B027A0079147D057C17786991
:1023AF0012081D158115817406900014F07F027BB1
:1023BF00027A007914124907021DDF7F017B057A2B
:1023CF00167945124907900104E0FAA3E0BA000319
:1023DF00B464005009900104E4F0A37464F0E52E96
:1023EF00B40120900104E0B40006A3E0B46401D36B
:1023FF004011900105E0249CFB900104E034FFF0B4
:08240F00A3EBF0E52EB4020678
:102417001249A6E4FF22E52EB4031F900104E0B59C
:102427002B05A3E0B52C005011900105E02464FBB7
:10243700900104E03400F0A3EBF0900104E0C0E069
:10244700A3E0C0E07B027A0079147D057C177869E8
:1024570012081D158115817406900014F07F027B08
:0B246700027A007914124907021DDF01
:102472008F27E4F528752901F52A752B10AE2AAFAE
:102482002B124A338E2C8F2DE52B2401FFE4352AA3
:10249200FE124A33EF900033F0E52B2402FFE435BD
:1024A2002AFE124A33EE900028F0A3EFF0E52B2427
:1024B20003FFE4352AFE124A33EF90002AF012009D
:0124C2000316
:1024C3001249B98F2EE52714600E14600B146008AF
:0824D300147003022D5080E893
:1024DB00E527B40117C028C0297B027A0079367D25
:1024EB00057C17787912081D15811581E527B40233
:1024FB0017C028C0297B027A0079367D057C1778B6
:10250B008B12081D15811581E527B40317C028C050
:10251B00297B027A0079367D057C17789D12081D80
:10252B0015811581E52EB4010280030225BEE52835
:0B253B00B40006E529B40001D340788D
:10254600E529152970021528E528B40006E529B401
:052556000001D3405D0F
:10255B00E52924FFFFE52834FFFEE4FC7D0A120188
:10256B0041EF2410F52BE43EF52AAE2AAF2B124A8D
:10257B00338E2C8F2DE52B2401FFE4352AFE124AD6
:10258B0033EF900033F0E52B2402FFE4352AFE12E3
:10259B004A33EE900028F0A3EFF0E52B2403FFE481
:0D25AB00352AFE124A33EF90002AF0800618
:1025B800E4F52875290BE52EB402028003022B30BE
:1025C800E529640B45287003E4FF22E527B40102DE
:0525D800800302271939
:1025DD00E5292400FBE5283455F5F0E52CB5F0028E
:0F25ED0080030226D5E52DB5030280030226D513
:1025FC007F017B057A1779AF124907C028C0297B68
:10260C00027A0079367D057C1778C012081D158179
:10261C0015817F027B027A007936124907E529245D
:10262C00FFFFE52834FFFEE4FC7D0A120141EF2494
:10263C0010F52BE43EF52AE52B2401FFE4352AFEA8
:10264C00124A33EF900106F0E52B2402FFE4352A01
:10265C00FE124A33EE9000FBF0A3EFF0E52B2403BF
:10266C00FFE4352AFE124A33EF9000FDF0E52B24EF
:10267C0004FFE4352AFE124A33EE900102F0A3EF78
:10268C00F0E52B2405FFE4352AFE124A33EE9001C7
:10269C0004F0A3EFF0E52B2406FFE4352AFE124AE2
:1026AC0033EE900107F0A3EFF0124AA3E4FE7F0E85
:1026BC00124AF6E4FE7F0EAC28AD29124A05124BE5
:0926CC00191249A6D204E4FF2210
:1026D5001249A67F017B057A1779D2124907C028CE
:1026E500C0297B027A0079367D057C1778E31208CC
:1026F5001D158115817F027B027A00793612490703
:10270500E4FE7F6412498E1249A67E057FDC1249DC
:0E2715008EE4FF22E527B40202800302297A37
:10272300E5292400FBE5283455F5F0E52CB5F00246
:0F273300800302288EE52DB50302800302288E55
:102742007B057A1779F5127ABFEF640160030229DB
:012752007A0C
:102753007F017B057A187906124907C028C0297BB7
:10276300027A0079367D057C18781712081D1581C9
:1027730015817F027B027A007936124907124AA338
:10278300E52924FFFFE52834FFFEE4FC7D0A12015E
:1027930041EF2410F52BE43EF52AAE2AAF2B124A63
:1027A300F6E52B2401FFE4352AFE124AF6E52B2435
:1027B30002FFE4352AFE124AF6E52B2403FFE43533
:1027C3002AFE124AF6E52B2404FFE4352AFE124AB8
:1027D300F6E52B2405FFE4352AFE124AF6E52B2401
:1027E30006FFE4352AFE124AF6AE2AAF2BE529246A
:1027F30000FDE5283455FC124A05E52B2401FFE4CE
:10280300352AFE900106E0FD7C00124A05E52B24E3
:1028130002FFE4352AFE9000FBE0FCA3E0FD124A30
:1028230005E52B2403FFE4352AFE9000FDE0FD7C43
:1028330000124A05E52B2404FFE4352AFE90010229
:10284300E0FCA3E0FD124A05E52B2405FFE4352A4D
:10285300FE900104E0FCA3E0FD124A05E52B2406EB
:10286300FFE4352AFE900107E0FCA3E0FD124A05D0
:10287300E4FE7F0E124AF6E4FE7F0EAC28AD291269
:0B2883004A05124B191249A6E4FF227F
:10288E007F017B057A187906124907C028C0297B7B
:10289E00027A0079367D057C18781712081D15818D
:1028AE0015817F027B027A007936124907124AA3FC
:1028BE00E52924FFFFE52834FFFEE4FC7D0A120122
:1028CE0041EF2410F52BE43EF52AAE2AAF2BE52975
:1028DE002400FDE5283455FC124A05E52B2401FFA2
:1028EE00E4352AFE900106E0FD7C00124A05E52B38
:1028FE002402FFE4352AFE9000FBE0FCA3E0FD126B
:10290E004A05E52B2403FFE4352AFE9000FDE0FD89
:10291E007C00124A05E52B2404FFE4352AFE9001C3
:10292E0002E0FCA3E0FD124A05E52B2405FFE43589
:10293E002AFE900104E0FCA3E0FD124A05E52B24DB
:10294E0006FFE4352AFE900107E0FCA3E0FD124AE3
:10295E0005E4FE7F0E124AF6E4FE7F0EAC28AD298A
:10296E00124A05124B191249A6E4FF22E527B403B9
:06297E00028003022B3071
:10298400E5292400FBE5283455F5F0E52CB5F002E3
:0F2994008003022A72E52DB503028003022A7226
:1029A3007B057A187929127ABFEF64016003022B41
:0129B30030F3
:1029B4007F017B057A18793A124907C028C0297B20
:1029C400027A0079367D057C1778C012081D1581BE
:1029D40015817F027B027A007936124907124AA3D5
:1029E400E52924FFFFE52834FFFEE4FC7D0A1201FB
:1029F40041EF2410F52BE43EF52AAE2AAF2B124A00
:102A0400F6E52B2401FFE4352AFE124AF6E52B24D1
:102A140002FFE4352AFE124AF6E52B2403FFE435CF
:102A24002AFE124AF6E52B2404FFE4352AFE124A54
:102A3400F6E52B2405FFE4352AFE124AF6E52B249D
:102A440006FFE4352AFE124AF6E52B2407FFE43597
:102A54002AFE124AF6E4FE7F0E124AF6E4FDFEFC5C
:0E2A64007F0E124A05124B191249A6E4FF22FA
:102A72007F017B057A18793A124907C028C0297B61
:102A8200027A0079367D057C1778C012081D1581FF
:102A920015817F027B027A007936124907124AA316
:102AA200E52924FFFFE52834FFFEE4FC7D0A12013C
:102AB20041EF2410F52BE43EF52AAE2AAF2B124A41
:102AC200F6E52B2401FFE4352AFE124AF6E52B2413
:102AD20002FFE4352AFE124AF6E52B2403FFE43511
:102AE2002AFE124AF6E52B2404FFE4352AFE124A96
:102AF200F6E52B2405FFE4352AFE124AF6E52B24DF
:102B020006FFE4352AFE124AF6E52B2407FFE435D8
:102B12002AFE124AF6E4FE7F0E124AF6E4FDFEFC9D
:102B22007F0E124A05124B191249A6E4FF22E52E26
:102B3200B403028003022BC4E528B40005E529B4DE
:072B42000C004003022BC44C
:102B49000529E52970020528640C45287006E4F575
:102B590028752901E528B40005E529B40B00505B67
:102B6900E52924FFFFE52834FFFEE4FC7D0A120174
:102B790041EF2410F52BE43EF52AAE2AAF2B124A79
:102B8900338E2C8F2DE52B2401FFE4352AFE124AC2
:102B990033EF900033F0E52B2402FFE4352AFE12CF
:102BA9004A33EE900028F0A3EFF0E52B2403FFE46D
:102BB900352AFE124A33EF90002AF0E529640B45C5
:032BC9002870155C
:102BCC007B027A0079367D057C18784B12081D74CF
:102BDC0006900036F07F017B027A007936124907A5
:102BEC00E52EB404037F0422E5292400FBE52834F8
:102BFC0055F5F0E52CB5F0028003022D13E52DB54B
:072C0C0003028003022D13F7
:102C1300900033E0601514603C146062147003028A
:0B2C23002CAA147003022CD3022CFA20
:102C2E00900028E0C0E0A3E0C0E0A3E0FBE4C0E039
:102C3E00C0037B027A0079367D057C18785C120819
:102C4E001D74FC2581F581022CFA900028E0C0E06D
:102C5E00A3E0C0E0A3E0FBE4C0E0C0037B027A0087
:102C6E0079367D057C18786E12081D74FC2581F569
:102C7E00818079900028E0C0E0A3E0C0E0A3E0FBF3
:102C8E00E4C0E0C0037B027A0079367D057C1878BB
:102C9E008012081D74FC2581F5818050900028E07B
:102CAE00C0E0A3E0C0E0A3E0FBE4C0E0C0037B0211
:102CBE007A0079367D057C18789312081D74FC25F0
:102CCE0081F5818027900028E0C0E0A3E0C0E0A35A
:102CDE00E0FBE4C0E0C0037B027A0079367D057C20
:102CEE001878A612081D74FC2581F5819000FDE070
:092CFE00600790010CE0B4011B19
:0C2D0700742090003CF07441A3F0800F99
:102D13007B027A0079367D057C1878B912081D7418
:102D230006900036F0E528B40005E529B40B005001
:102D33000E7F027B027A007936124907022E5A7FF0
:102D4300027B057A1879CA1249070224C37B057AE4
:0E2D53001879DB127ABFEF64016003022E5A7A
:102D61007F017B057A1879EC1249077F027B057A8E
:102D71001879FD124907124AA3124AB9E4FE7F6489
:102D810012498EE4FDFEFF7C01124A05E4FE7F013B
:102D910090010CE0FD7C00124A05E4FE7F029001E7
:102DA10016E0FD7C00124A05E4FE7F0390011AE063
:102DB100FD7C00124A05E4FE7F0490011BE0FD7CCE
:102DC10000124A05E4FE7F05900113E0FCA3E0FD3B
:102DD100124A05E4FE7F06900109E0FCA3E0FD1222
:102DE1004A05E4FE7F0790011CE0FCA3E0FD124AC6
:102DF10005E4FE7F08900110E0FCA3E0FD124A0506
:102E0100E4FE7F09900117E0FD7C00124A05E4FE13
:102E11007F0A900118E0FD7C00124A05E4FE7F0B59
:102E2100900119E0FD7C00124A05E4FE7F0C90013F
:102E31000DE0FD7C00124A05E4FE7F0D90010EE0DD
:102E4100FCA3E0FD124A05E4FDFEFC7F0E124A05DB
:0C2E5100124B191249A6E4FF220224C310
:052E5D008F27120003A5
:102E62001249B98F28E528B404037F0422E5271408
:102E72006014147003022F19147003022FDA1470F5
:062E82000302305280DA69
:102E88007F017B057A19790E12490790010CE0B48D
:102E980001117B027A00794A7D057C19781F120896
:102EA8001D800F7B027A00794A7D057C19783012E3
:102EB800081D740690004AF07F027B027A00794A66
:0E2EC800124907E52864016005E528B40311EE
:102ED60090010CE0B40104E4F08006740190010C4A
:0B2EE600F0E528B4020280030230DE99
:072EF100900115E0B4011B84
:102EF800124AA3E4FE7F01124AF6E4FE7F01900124
:102F08000CE0FD7C00124A05124B191249A6E4FF99
:102F1800227F017B057A197941124907E528B40116
:012F28001593
:102F2900900116E0B40101D34005E014F080067465
:0A2F390003900116F0E528B4022809
:072F4300900115E0B4011B31
:102F4A00124AA3E4FE7F02124AF6E4FE7F029001CF
:102F5A0016E0FD7C00124A05124B191249A6E4FF3D
:062F6A0022E528B4031467
:102F7000900116E0B403005005E004F080067401EF
:102F8000900116F0900116E0B4010F7B027A0079EF
:102F90004A7D057C19785212081D900116E0B40292
:102FA0000F7B027A00794A7D057C19786312081D2F
:102FB000900116E0B4030F7B027A00794A7D057C0C
:102FC00019787412081D740690004AF07F027B0283
:102FD0007A00794A124907022E627F017B057A192D
:102FE000798512490790010BE0FBE4C0E0C0037B48
:102FF000027A00794A7D057C1578F112081D158149
:103000001581740690004AF07F027B027A00794AAB
:10301000124907E528B4011090010BE0B40101D377
:0D302000400690010BE014F0E528B4020614
:10302D001249A6E4FF22E528B4030280030230DE34
:10303D0090010BE0B40A0040030230DE90010BE07A
:10304D0004F0022E627F017B057A197996124907E9
:10305D0090011AE0B401117B027A00794A7D057C5A
:10306D001978A712081D800F7B027A00794A7D0519
:10307D007C1978B812081D740690004AF07F027B07
:10308D00027A00794A124907E52864016005E528AE
:03309D00B4031168
:1030A00090011AE0B40104E4F08006740190011A62
:0630B000F0E528B402283F
:0730B600900115E0B4011BBD
:1030BD00124AA3E4FE7F03124AF6E4FE7F03900159
:1030CD001AE0FD7C00124A05124B191249A6E4FFC5
:0430DD0022022E623B
:0630E1007524011200033A
:1030E7001249B98F25E52514601214602214700364
:0C30F7000231951470030231A50231A8CB
:10310300E524B40101D3400515240231A875240533
:083113000231A8E524B4050611
:06311B00120003E4FF2294
:10312100E52464026005E524B40329900106E0B4B6
:053131000101D3401F65
:103136007F017B057A1A79511249077F027B057A4E
:103146001A79621249077E077FD012498E803BE5C5
:0C31560024B40327900116E06401601F00
:103162007F017B057A1A79511249077F027B057A22
:0F3172001A79731249077E077FD012498E800F9A
:10318100AF24122E5D8F26E526B404037F0422129C
:1031910000038013E524B40500500405248008755C
:1031A100240180037F0422E524146018146058145C
:1031B10070030232661470030232D41470030233B6
:0431C100160230E7DB
:1031C5007B027A0079727D057C1A788412081D7459
:1031D50006900072F07F017B027A0079721249072E
:1031E50090010CE0B4010E7F027B057A1A799512E5
:1031F50049070233417F027B057A1A79A6124907EE
:103205000230E77B027A0079727D057C1A78B71265
:10321500081D7406900072F07F017B027A007972B6
:10322500124907900116E0B4010B7F027B057A1A5B
:1032350079C8124907900116E0B4020B7F027B059D
:103245007A1A79D9124907900116E0B4030280036E
:103255000233417F027B057A1A79EA124907023067
:10326500E77B027A0079727D057C1A78FB12081DCE
:103275007406900072F07F017B027A007972124920
:1032850007900106E0B40101D35008900116E064EF
:103295000160117B027A0079727D057C1B780C1226
:1032A500081D801D90010BE0FBE4C0E0C0037B021C
:1032B5007A0079727D057C1578F112081D15811546
:1032C500817F027B027A0079721249070230E77B1F
:1032D500027A0079727D057C1B781D12081D740623
:1032E500900072F07F017B027A0079721249079093
:1032F500011AE0B4010D7F027B057A1B792E124974
:103305000780397F027B057A1B793F124907023016
:10331500E77B027A0079727D057C1B785012081DC7
:103325007406900072F07F017B027A00797212496F
:0F333500077F027B057A1879CA1249070230E731
:06334400E4F52112000374
:10334A001249B98F22E52214600C14601C14700310
:06335A000233E90233F723
:10336000E521B40001D3400515210233F77521038F
:103370000233F7E521600B14602714604714606383
:02338000807556
:0D3382001202668F23120003E523B40458E5
:10338F001249A630800320814FE4FE7F6412498EDC
:0F339F0080F11206018F23120003E523B40412FC
:1033AE001249A6308003208109E4FE7F6412498E03
:1033BE0080F1300424221230E18F23120003E52322
:0333CE00B404162E
:1033D1001249A630800320810DE4FE7F6412498EDC
:1033E10080F112000322800EE521B4030050040590
:1033F100218003E4F521E521600B14601914602795
:0534010014603580425B
:103406007B027A0079867D057C1B786112081D8017
:10341600317B027A0079867D057C1B787212081D45
:1034260080207B027A0079867D057C1B78831208D2
:103436001D800F7B027A0079867D057C1B789412AD
:10344600081D7406900086F07F017B027A0079865B
:103456001249077B027A0079867D057C1A7840122C
:10346600081D740590008AF004A3F07F027B027A9F
:0934760000798612490702334A6D
:10347F007F017B057A1B79A51249077F027B057AAD
:10348F001B79B61249077E057FDC12498E7F017BBF
:10349F00057A1B79C71249077F027B057A1B79D8FA
:1034AF001249077E057FDC12498EE4F521120003D5
:1034BF001249B98F22E52214600814601614602691
:0234CF00803249
:1034D100E521B40001D340041521802675210A801D
:0634E10021E521B40A04FC
:0434E70012000322AA
:1034EB00AF2112393C120003800EE521B40A0050C3
:1034FB000405218003E4F521E521B40B0040030210
:10350B003939FA232A903514730235370235820282
:10351B0035CD0236180236630236CF02373B0237FF
:0C352B00860237D102387102390E808808
:103537007B027A00799A7D057C1B78E912081D7455
:103547000690009AF07F017B027A00799A12490768
:1035570090010EE0C0E0A3E0C0E07B027A00799A18
:103567007D057C1B78FA12081D158115817F027B6A
:10357700027A00799A1249070234BF7B027A0079EE
:103587009A7D057C1C780A12081D740690009AF033
:103597007F017B027A00799A124907900109E0C0FE
:1035A700E0A3E0C0E07B027A00799A7D057C1B7876
:1035B700FA12081D158115817F027B027A00799A1C
:1035C7001249070234BF7B027A00799A7D057C1C79
:1035D700781B12081D740690009AF07F017B027A0F
:1035E70000799A124907900119E0FBE4C0E0C00393
:1035F7007B027A00799A7D057C1C782C12081D15B0
:103607008115817F027B027A00799A124907023479
:10361700BF7B027A00799A7D057C1C783D12081DD4
:10362700740690009AF07F017B027A00799A12491A
:103637000790010DE0FBE4C0E0C0037B027A00794C
:103647009A7D057C1C782C12081D158115817F0237
:103657007B027A00799A1249070234BF7B027A000B
:10366700799A7D057C1C784E12081D740690009A85
:10367700F07F017B027A00799A124907E4FCFD90FA
:103687000113E0FEA3E0FF121491C004C005C006B9
:10369700C0077C6F7D127E837F3A12112CC004C055
:1036A70005C006C0077B027A00799A7D057C1C78E5
:1036B7005F12081D74FC2581F5817F027B027A0069
:1036C700799A1249070234BF7B027A00799A7D05FD
:1036D7007C1C787112081D740690009AF07F017B9C
:1036E700027A00799A124907E4FCFD900110E0FE86
:1036F700A3E0FF121491C004C005C006C0077C6F89
:103707007D127E837F3A12112CC004C005C006C00B
:10371700077B027A00799A7D057C1C785F12081D69
:1037270074FC2581F5817F027B027A00799A124920
:10373700070234BF7B027A00799A7D057C1C788268
:1037470012081D740690009AF07F017B027A0079B7
:103757009A124907900117E0FBE4C0E0C0037B021F
:023767007A00E6
:10376900799A7D057C1C789312081D158115817F36
:10377900027B027A00799A1249070234BF7B027AE6
:1037890000799A7D057C1C78A612081D74069000A4
:103799009AF07F017B027A00799A12490790011801
:1037A900E0FBE4C0E0C0037B027A00799A7D057CE6
:1037B9001C789312081D158115817F027B027A00FE
:1037C900799A1249070234BF7B027A00799A7D05FA
:1037D9007C1C78B712081D740690009AF07F017B53
:1037E900027A00799A12490790011CE0FEA3E0FFD2
:1037F900E4FCFD121491C004C005C006C00774CDD5
:10380900FC14FDFE743DFF12112C8C238D248E2592
:103819008F2690011BE0FF124C15E4FCFD12149158
:10382900C004C005C006C007AC23AD24AE25AF2631
:10383900121288C004C005C006C00790011BE0FB36
:10384900E4C0E0C0037B027A00799A7D057C1C788C
:10385900C812081D74FA2581F5817F027B027A005E
:10386900799A1249070234BF7B027A00799A7D0559
:103879007C1C78DB12081D740690009AF07F017B8E
:10388900027A00799A12490790011CE0FEA3E0FF31
:10389900E4FCFD121491C004C005C006C00774CD34
:1038A900FC14FDFE743DFF12112C8C238D248E25F2
:1038B9008F267F05124C15E4FCFD121491C004C03B
:1038C90005C006C007AC23AD24AE25AF2612128869
:1038D900C004C005C006C00790011CE0C0E0A3E019
:1038E900C0E07B027A00799A7D057C1C78EC12088D
:1038F9001D74FA2581F5817F027B027A00799A127B
:1039090049070234BF7B027A00799A7D057C1C78CD
:10391900FC12081D740690009AF07F017B027A0060
:10392900799A1249077F027B057A1879CA124907E1
:033939000234BF96
:05393C008F27120003BB
:103941001249B98F28E527B40A0040030240ECFA76
:10395100232A90395773023977023A30023AE90241
:103961003B84023C2E023D08023DE2023E7A023FC8
:0639710012023FF880CABB
:103977007F017B057A1D790D12490790010EE0C082
:10398700E0A3E0C0E07B027A0079AE7D057C1B787E
:10399700FA12081D1581158174069000AEF07F029A
:1039A7007B027A0079AE124907E528B4012090011D
:1039B7000EE0B40306A3E0B4E801D3401190010F71
:1039C700E024F6FB90010EE034FFF0A3EBF0E528CE
:0339D700B4022710
:0739DA00900115E0B4011C8F
:1039E100124AA3E4FE7F0D124AF6E4FE7F0D900118
:1039F1000EE0FCA3E0FD124A05124B191249A62262
:103A0100E528B4030280030240EC90010EE0B40704
:103A110005A3E0B4D00040030240EC90010FE02484
:103A21000AFB90010EE03400F0A3EBF00239417F74
:103A3100017B057A1D791E124907900109E0C0E05A
:103A4100A3E0C0E07B027A0079AE7D057C1B78FAA9
:103A510012081D1581158174069000AEF07F027B5E
:103A6100027A0079AE124907E528B40120900109D4
:103A7100E0B40306A3E0B4E801D3401190010AE0E9
:103A810024F6FB900109E034FFF0A3EBF0E528B444
:023A910002270A
:073A9300900115E0B4011CD5
:103A9A00124AA3E4FE7F06124AF6E4FE7F0690016C
:103AAA0009E0FCA3E0FD124A05124B191249A622AD
:103ABA00E528B4030280030240EC900109E0B40750
:103ACA0005A3E0B4D00040030240EC90010AE024D0
:103ADA000AFB900109E03400F0A3EBF00239417FC0
:103AEA00017B057A1D792F124907900119E0FBE441
:103AFA00C0E0C0037B027A0079AE7D057C1C782C7D
:103B0A0012081D1581158174069000AEF07F027BA4
:103B1A00027A0079AE124907E528B401109001191A
:103B2A00E0B41E01D34006900119E014F0E528B470
:023B3A00022661
:073B3C00900115E0B4011B2C
:103B4300124AA3E4FE7F0B124AF6E4FE7F0B9001B8
:103B530019E0FD7C00124A05124B191249A622E511
:103B630028B4030280030240EC900119E0FB7A00C1
:103B7300B4F00040030240EC900119E004F0023974
:103B8300417B027A0079AE7D057C1D784012081DC9
:103B93007F017B027A0079AE12490790010DE0FBA9
:103BA300E4C0E0C0037B027A0079AE7D057C1C781B
:103BB3002C12081D1581158174069000AEF07F024A
:103BC3007B027A0079AE124907E528B4011090010F
:103BD3000DE0B41E01D3400690010DE014F0E5287A
:033BE300B4022603
:073BE600900115E0B4011B82
:103BED00124AA3E4FE7F0C124AF6E4FE7F0C90010C
:103BFD000DE0FD7C00124A05124B191249A622E573
:103C0D0028B4030280030240EC90010DE0FB7A0022
:103C1D00B4F00040030240EC90010DE004F00239D5
:103C2D00417F017B057A1D7951124907900113E0FF
:103C3D00FEA3E0FFE4FCFD121491C004C005C00614
:103C4D00C0077C6F7D127E837F3A12112CC004C099
:103C5D0005C006C0077B027A0079AE7D057C1D7814
:103C6D006212081D74FC2581F58174069000AEF07A
:103C7D007F027B027A0079AE124907E528B4012054
:103C8D00900113E0B40606A3E0B44001D3401190B7
:103C9D000114E024F6FB900113E034FFF0A3EBF0E8
:053CAD00E528B4022728
:073CB200900115E0B4011CB4
:103CB900124AA3E4FE7F05124AF6E4FE7F0590014D
:103CC90013E0FCA3E0FD124A05124B191249A62282
:103CD900E528B4030280030240EC900113E0B40725
:103CE90005A3E0B46C0040030240EC900114E02409
:103CF9000AFB900113E03400F0A3EBF00239417F95
:103D0900017B057A1D7973124907900110E0FEA322
:103D1900E0FFE4FCFD121491C004C005C006C00711
:103D29007C6F7D127E837F3A12112CC004C005C0BE
:103D390006C0077B027A0079AE7D057C1D78621288
:103D4900081D74FC2581F58174069000AEF07F0290
:103D59007B027A0079AE124907E528B40120900167
:103D690010E0B40106A3E0B4F401D34011900111AD
:103D7900E024F6FB900110E034FFF0A3EBF0E52816
:033D8900B402275A
:073D8C00900115E0B4011CD9
:103D9300124AA3E4FE7F08124AF6E4FE7F0890016C
:103DA30010E0FCA3E0FD124A05124B191249A622AA
:103DB300E528B4030280030240EC900110E0B40450
:103DC30005A3E0B4B00040030240EC900111E024ED
:103DD3000AFB900110E03400F0A3EBF00239417FBD
:103DE300017B057A1D7984124907900117E0FBE4F2
:103DF300C0E0C0037B027A0079AE7D057C1D789517
:103E030012081D1581158174069000AEF07F027BA8
:103E1300027A0079AE124907E528B4011090011720
:103E2300E0B40501D34006900117E014F0E528B48F
:023E3300022665
:073E3500900115E0B4011B30
:103E3C00124AA3E4FE7F09124AF6E4FE7F099001C0
:103E4C0017E0FD7C00124A05124B191249A622E517
:103E5C0028B4030280030240EC900117E0B419006F
:103E6C0040030240EC900117E004F00239417F015D
:103E7C007B057A1D79A7124907900118E0FBE4C075
:103E8C00E0C0037B027A0079AE7D057C1D7895122B
:103E9C00081D1581158174069000AEF07F027B021F
:103EAC007A0079AE124907E528B40110900118E0A8
:103EBC00B40301D34006900118E014F0E528B402D5
:013ECC0026CF
:073ECD00900115E0B4011B98
:103ED400124AA3E4FE7F0A124AF6E4FE7F0A900126
:103EE40018E0FD7C00124A05124B191249A622E57E
:103EF40028B4030280030240EC900118E0B40A00E5
:103F040040030240EC900118E004F00239417F01C3
:103F14007B057A1D79B812490790011CE0FEA3E0E5
:103F2400FFE4FCFD121491C004C005C006C0077470
:103F3400CDFC14FDFE743DFF12112C9000C2120042
:103F4400E390011BE0FF124C15E4FCFD121491C038
:103F540004C005C006C0079000C2121285C004C088
:103F640005C006C00790011BE0FBE4C0E0C0037B72
:103F7400027A0079AE7D057C1C78C812081D74FA9B
:103F84002581F58174069000AEF07F027B027A00F1
:103F940079AE124907E528B4011090011BE0B40082
:0F3FA40001D3400690011BE014F0E528B402267B
:073FB300900115E0B4011BB1
:103FBA00124AA3E4FE7F04124AF6E4FE7F0490014B
:103FCA001BE0FD7C00124A05124B191249A622E594
:103FDA0028B4030280030240EC90011BE0B4040001
:103FEA0040030240EC90011BE004F00239417F01DA
:103FFA007B057A1D79C912490790011CE0FEA3E0EE
:10400A00FFE4FCFD121491C004C005C006C0077489
:10401A00CDFC14FDFE743DFF12112C9000C212005B
:10402A00E37F05124C15E4FCFD121491C004C0058F
:10403A00C006C0079000C2121285C004C005C0069F
:10404A00C00790011CE0C0E0A3E0C0E07B027A0058
:10405A0079AE7D057C1C78EC12081D74FA2581F571
:10406A008174069000AEF07F027B027A0079AE126C
:10407A004907E528B4011E90011CE0B40706A3E035
:10408A00B4D001D3400F90011DE014F0F490011C4C
:0A409A007003E014F0E528B40227DB
:0740A400900115E0B4011CBE
:1040AB00124AA3E4FE7F07124AF6E4FE7F07900153
:1040BB001CE0FCA3E0FD124A05124B191249A62283
:1040CB00E528B4031C90011CE0B40B05A3E0B4B8C5
:1040DB0000500E90011DE004F090011C7003E004F1
:0440EB00F002394165
:1040EF008E218F228D238D07120771EE9000E6F03F
:1040FF00A3EFF0E4FDFC9000DAF090011CE0FEA3CA
:10410F00E0FF1214919000DC1200E3E4FCFD90013B
:10411F0007E0FEA3E0FF121491C004C005C006C063
:10412F00077C6F7D127E837F3A12112CC004C0056D
:10413F00C006C0079000FDE0FF7E00E433E45001AD
:10414F0014FCFD12145412112CC004C005C006C07B
:10415F00079000DC121129121495EE9000E2F0A3E3
:10416F00EFF0E52324FD70030243C51470030243EF
:09417F00C524FE60041460012255
:10418800AF23120771EE9000E0F0A3EFF0701890E3
:1041980000E0E070129000E6E0FAA3E0FB9000E097
:1041A800EAF0A3EBF080109000E0E0FAA3E0FB90C7
:1041B80000E6EAF0A3EBF0E4FCFDAE21AF22121416
:1041C80091C004C005C006C00774CDFC14FDFE7480
:1041D8003CFF12112C121495EE9000E4F0A3EFF0BE
:0A41E800E523B406028003024277CB
:0E41F2009000DBE0F5F090012DE065F06077C5
:10420000E09000DBF07B027A0079C67D057C0778C0
:104210003D12081D74069000C6F07F017B027A00F3
:1042200079C6124907E5FEFF7E00E4FC7D641201B9
:1042300041E4FC7DFF120155C006C0077B027A00F5
:1042400079C67D057C07784E12081D15811581857C
:1042500021248522257B027A0079C69000E0E0FCCB
:10426000A3E0FD1246E274259000D5F07F027B02A8
:104270007A0079C61249079000E0E0FAA3E0FBEA71
:10428000FEEBFF9000E5E0F8E522C398FD9000E426
:10429000E0FBE5219BFCF5F0EAB5F004EFB5050085
:1042A000500CE5FEFB7A00B4F200500205FE9000CF
:1042B000E0E0FAA3E0FB9000E5E02522FD9000E4B9
:1042C000E03521FCF5F0EAB5F005EBB50501D3408A
:1042D0000AE5FEB40001D3400215FE9000E0E0FCC8
:1042E000A3E0FD9000E5E0FAE522C39AFB9000E42C
:1042F000E0F8E52198FAF5F0ECB5F004EDB503002F
:10430000401EA3E02522FB9000E4E03521FAF5F001
:10431000ECB5F005EDB50301D350058C068D0722F1
:10432000E5FEB40101D3400AE5FEFB7A00B4F100DA
:1043300040099000E0E0FEA3E0FF22900106E0B417
:054340000101D340491A
:104345001207B1E4FCFD121491C004C005C006C0FB
:1043550007E4FCFD9000E2E0FEA3E0FF121491C02B
:1043650004C005C006C0079000DC12009CE4FEFCFA
:10437500FD743FFF12112C120FCC121522BF01093B
:104385009000E0E0FEA3E0FF229000DAE004F0E513
:1043950023B40710E0B40801D340099000E0E0FE23
:1043A500A3E0FF22E523B4070280030241883080A1
:1043B500063081030241889000E0E0FEA3E0FF2281
:1043C500AF23120771EE9000E0F0A3EFF0701890A4
:1043D50000E0E070129000E6E0FAA3E0FB9000E058
:1043E500EAF0A3EBF080109000E0E0FAA3E0FB9088
:1043F50000E6EAF0A3EBF0E4FCFDAE21AF221214D7
:1044050091C004C005C006C00774CDFC14FDFE7440
:104415003CFF12112C121495EE9000E4F0A3EFF07E
:0A442500E523B4030280030244B44F
:0E442F009000DBE0F5F090012DE065F0607785
:10443D00E09000DBF07B027A0079C67D057C077881
:10444D006012081D74069000C6F07F017B027A0091
:10445D0079C6124907E5FDFF7E00E4FC7D6412017B
:10446D0041E4FC7DFF120155C006C0077B027A00B6
:10447D0079C67D057C07784E12081D15811581853D
:10448D0021248522257B027A0079C69000E0E0FC8C
:10449D00A3E0FD1246E274259000D5F07F027B0269
:1044AD007A0079C61249079000E0E0FAA3E0FB908C
:1044BD0000E5E0F8E522C398FD9000E4E0F8E52181
:1044CD0098FCF5F0EAB5F004EBB50500500CE5FDF0
:1044DD00FB7A00B4F200500205FD9000E0E0FAA373
:1044ED00E0FB9000E5E02522FD9000E4E03521FCA5
:1044FD00F5F0EAB5F005EBB50501D3400AE5FDB4DD
:10450D000001D3400215FD9000E0E0FCA3E0FD901A
:10451D0000E5E0FAE522C39AFB9000E4E0F8E5211E
:10452D0098FAF5F0ECB5F004EDB50300401EA3E0EC
:10453D002522FB9000E4E03521FAF5F0ECB5F0050D
:10454D00EDB50301D350058C068D0722E5FDB401B1
:10455D0001D3400AE5FDFB7A00B4F100400990005B
:10456D00E0E0FEA3E0FF229000DAE004F0E523B4E2
:10457D000410E0B40801D340099000E0E0FEA3E090
:10458D00FF22E523B4040280030243C530800630C8
:0E459D0081030243C59000E0E0FEA3E0FF2290
:1045AB008E218F221207B1EE9000E8F0A3EFF0E41A
:1045BB00FCFD90011CE0FEA3E0FF1214919000EAB9
:1045CB001200E31207B1EE9000EEF0A3EFF07018BB
:1045DB009000EEE070129000E8E0FAA3E0FB900090
:1045EB00EEEAF0A3EBF080109000EEE0FAA3E0FB14
:1045FB009000E8EAF0A3EBF09000EA12009C7C0A32
:10460B007DD77EA37F3B12112C1214959000F0EEF8
:10461B00F0A3EFF09000EEE0FCA3E0FD9000F1E0E2
:10462B00FAE522C39AFB9000F0E0F8E52198FAF541
:10463B00F0ECB5F004EDB50300500CE5FEFB7A0091
:10464B00B4F200500205FE9000EEE0FCA3E0FD90FA
:10465B0000F1E02522FB9000F0E03521FAF5F0ECBB
:10466B00B5F005EDB50301D3400AE5FEB40001D367
:10467B00400215FE9000EEE0FCA3E0FD9000F1E09F
:10468B00FAE522C39AFB9000F0E0F8E52198FAF5E1
:10469B00F0ECB5F004EDB50300401EA3E02522FBC2
:1046AB009000F0E03521FAF5F0ECB5F005EDB5032F
:1046BB0001D350058C068D0722E5FE64016006E5EB
:1046CB00FE64F170099000EEE0FEA3E0FF22900083
:0746DB00EEE0FEA3E0FF2268
:1046E2008B268A2789288C298D2AE4FCFDAE29AFE6
:1046F2002A121491C004C005C006C007E4FCFD7470
:10470200C8FE7442FF12112CC004C005C006C007C7
:10471200E4FCFDAE24AF25121491121288121495F6
:104722008F2BAD26AC27A828AB26AA27A928E412EE
:04473200002A7F01D9
:1047360008E870010CEDFBECFAE8F9740112002AA6
:104746000FBF09EC08E870010CEDFBECFAE8F97410
:074756000212002A752C007D
:10475D00AF2C7E00E4FC7D0A1201418EF0B2F7749D
:0C476D0080B5F006E52BB50701D34041F4
:10477900AB26AA27A928740312002A0528E5287060
:10478900020527E52CB40800500CAB26AA27A92856
:10479900E412002A800BAB26AA27A9287403120069
:1047A9002AE52CB4090BAB26AA27A92874201200E4
:0947B9002A052CE52CB40A9C220F
:1047C20075FA0075EA0075DA0075FB0075EB007585
:1047D200DB0075FC0075EC0075DC0075FD0075ED05
:1047E2000075DD0075FE0075EE0075DE00C2DED2DA
:0A47F20093D294D295D296D297226A
:1047FC00C283E4FE7F641207D27F331207ED7F324F
:10480C001207ED7F281207ED7F0C1207ED7F0612C1
:0F481C0007ED7F011207ED7E017FF41207D22214
:10482B008F0553800FED54F04280D283E4FE7F322C
:10483B001207D2C28353800FEDC454F04280D2834F
:10484B00E4FE7F321207D2C2837E017FF41207D2BD
:01485B00223A
:10485C000E1F111111111F000E1F1111111F1F001E
:10486C000E1F11111F1F1F000E1F111F1F1F1F00D6
:10487C000E1F1F1F1F1F1F000002060E0602000046
:10488C0000080C0E0C080000001F1517111F00006B
:10489C00001F10101010101F001F00000000001F40
:1048AC00001F01010101011F001F1F1F1F1F1F1FE0
:1048BC000E1F11111F1F1F000002060E0602000022
:1048CC0000080C0E0C080000001F1517111F00002B
:1048DC008F21752240E52175F040A4F52175230048
:1048EC00AF221207EDE521252390485C93FF1207B8
:0B48FC00E505220523E523B440E62279
:104907008F358B368A378938EF14600A14600E1496
:064917006012146016227C
:10491D007F801207ED80137FC01207ED800C7FFFA3
:0D492D001207ED80057FFF1207ED753900C0
:10493A00AB36AA37A938120071FF1207E50538E528
:0D494A0038700205370539E539B410E42254
:0749570090011AE0B4011CFD
:03495E00752100C0
:10496100C2B5E4FE7F2812498ED2B5E4FE7F3C1227
:0A497100498E0521E521B405E72277
:07497B0090011AE0B4010BEA
:0C498200C2B5E4FE7F3C12498ED2B52283
:04498E00EE4F601375
:104992007B007A06DBFEDAFC7C06E4FDEF1F70EC9E
:0449A2001E80E92268
:0749A60090011AE0B4010BBF
:0C49AD00C2B57E037F2012498ED2B522D5
:1049B900E4F5352080037535012081037535022022
:1049C9008006208103753503E535600312497B3084
:0549D900800320812194
:1049DE00E4FE7F3212498EE50AB40F01D3400EE594
:0449EE0035B40206D4
:1049F200E4F50A7F0422AF3522050A80D9E4F50ADC
:034A0200AF3522AB
:104A05008C2F8D309000F27403F0A374E8F0D2A3DC
:104A1500EF2400F532EE3405F531AE31AF32124BED
:0E4A25002FAE2FAF30124B74124BB7C2A3222C
:104A33009000F27401F0A3742CF0D2A3EF2400F5DC
:104A430030EE3406F52FAE2FAF30124B2F124A5EE5
:0B4A53008E318F32C2A3AE31AF322291
:0F4A5E00E4F533F534F53575360FE53520E731DE
:104A6D00124BE1A2A0E4335401753700F538AB3891
:104A7D00AA37A836088005C333CA33CAD8F94534D6
:104A8D00F534EA4533F533E536153670CE153580F8
:064A9D00CAAE33AF342263
:104AA3009000F27403F0A374E8F0D2A37E047FC0F5
:064AB300124B2FC2A322EA
:104AB9009000F27403F0A374E8F0D2A37E047F801F
:094AC900124B2F124BB7C2A322BD
:104AD2008E088F099000F27403F0A374E8F0D2A359
:104AE2007E047F40124B2FAE08AF09124B74124B5B
:044AF200B7C2A32282
:104AF6009000F27403F0A374E8F0D2A3EF2400F55B
:104B060030EE3407F52FAE2FAF30124B2F124BB7C6
:034B1600C2A32215
:104B19009000F27403F0A374E8F0D2A37E04E4FFDA
:064B2900124B2FC2A32273
:0F4B2F008E338F34E4F53575360AE53520E733DC
:104B3E00AB34AA33E533A836088005C313CB13CBA9
:104B4E00D8F9EB5401753700F53864014537700418
:104B5E00D2A18002C2A1124BE1E536153670CC15FA
:064B6E003580C8C2A1223F
:0F4B74008E338F34E4F53575360FE53520E73392
:104B8300AB34AA33E533A836088005C313CB13CB64
:104B9300D8F9EB5401753700F538640145377004D3
:104BA300D2A18002C2A1124BE1E536153670CC15B5
:044BB3003580C8225F
:104BB700C2A39000F2E0FEA3E0FF124BFCD2A37465
:104BC700FFFAFB20A013EA6480B48004BB0001D382
:0A4BD7004007EB1B70ED1A80EA2284
:104BE100D2A29000F2E0FEA3E0FF124BFCC2A29021
:0B4BF10000F2E0FEA3E0FF124BFC22EC
:104BFC00E4FAFB8EF0EAB5F0068FF0EBB5F000505E
:094C0C00070BEB70EE0A80EB22AD
:104C15008F359000F51200EF00000000E49000F4DD
:014C2500F09E
:104C2600E4FE7FC81207D2AF35124C79EE9000F938
:104C3600F0A3EFF09000F512009CE4FCFD9000F963
:104C4600E0FEA3E0FF12012C9000F51200E39000B5
:104C5600F4E004F0648070C875F007A31200D71260
:104C660001179000F9EEF0A3EFF09000F9E0FEA333
:034C7600E0FF223A
:104C7900EF441823232354F8FFD2A40000D2A7003D
:074C890000C2A700007E0538
:104C9000C2A4EF30E704D2A68002C2A6EFC333FF5E
:104CA0000000D2A40000DEE8D2A6C2A40000D2A474
:0A4CB0000000C2A40000E4FF7E052E
:104CBA00EFC333FF30A5034401FFD2A40000C2A40E
:0D4CCA000000DEECEF540FFCE4FFFD7E085F
:104CD700EFC333FF30A5034401FFD2A40000C2A4F1
:0D4CE7000000DEECEF2DFFE43CFED2A72222
:104CF400C0E0C083C082C0D0C002C003758C877579
:0B4D04008AFF90012EE0B464005046CE
:104D0F00E004F0900100E0FAA3E0BA0004B400015F
:104D1F00D3400CE014F0F49001007003E014F09015
:064D2F00012EE0B4325F2A
:104D350090012DE070057401F08005E490012DF0DF
:104D450090012CE004F0B40401D34043E4F0803F2B
:104D5500E490012EF0A3E004F0A3E0FAA3E0BA008A
:104D650004B40001D3400CE014F0F490013070035A
:104D7500E014F0900134E0FAA3E0BA0004B40001B5
:104D8500D3400CE014F0F49001347003E014F0907B
:094D9500012FE0B43B01D34010F2
:104D9E00E4F0900133E004F09001327003E004F08F
:0D4DAE00D003D002D0D0D082D083D0E0322C
:104DBB0020202057454C434F4D4520544F20202059
:104DCB000020534D415254204348415247455220F5
:104DDB002000436F7079726967687420284329201B
:104DEB004279007777772E686F6262792D72632E26
:104DFB00636F6D0020496E697469616C204D656D40
:104E0B006F7279200020506C656173652057616962
:104E1B00742E2E2E200020202A2A204552524F522B
:104E2B00202A2A2020200020204D656D6F727920CA
:104E3B004661696C202020004C6F6164696E6720AD
:104E4B0042617474657279200046726F6D204C6FED
:104E5B00636174696F6E20253264004C6F61646905
:104E6B006E672044656661756C74200042617474D2
:104E7B0065727920496E666F2E2E2E200043686175
:104E8B00726765722066756E6374696F6E00697305
:104E9B002064697361626C65642E202020200044BD
:104EAB00697363682E2066756E6374696F6E20007C
:104EBB00202020202025326443202534646D416856
:104ECB000020204E6F20426174746572792020207F
:104EDB002000202025352E3266562025352E3266B1
:104EEB0056730053544F5020444953434841524743
:104EFB0045523F00204449534348415247452020E7
:104F0B002020202000202020576169742025336445
:104F1B00207365632E00205374617274204469738F
:104F2B0063686172676500202020202020202020EC
:104F3B002020202020202000202020202020202086
:104F4B0020252B34646D41680025352E32665620A2
:104F5B0025332E31664120253364730025352E32DF
:104F6B0066562025332E316641202533646D00258E
:104F7B00352E32665673202050574D202532642033
:104F8B000053544F5020434841524745523F202035
:104F9B00200020434841524745202020202020203C
:104FAB002020200020537461727420436861726763
:104FBB0065722020002046554C4C592043484152E5
:104FCB004745202020002044495343484152474540
:104FDB0020444F4E452000205553455220544552F6
:104FEB004D494E415445440020424154542E204FCC
:104FFB005645522D564F4C54002042415454204498
:10500B004953434F4E4E45435400204C4F5720536A
:10501B005550504C5920564F4C5400204449534343
:10502B00482E2020252B34646D41680020444953C1
:10503B0043482E54494D45202533646D0020434889
:10504B00415247452020252B34646D416800204395
:10505B0048472E54494D452020202533646D0020B0
:10506B0025352E326656702025352E326656652034
:10507B000020535550504C59202025352E32665662
:10508B007320002020204E6F202020202059657394
:04509B0020202000B1
:10509F007580FF7590FF75A0FF75B0FFE4FE7FFA76
:1050AF0012498E1247FC120003E4FF1248DC758987
:1050BF0001758C87758AFFD28C75A8821207C8126A
:1050CF0047C21207F5308007208104D2008002C248
:1050DF00007F017B057A4D79BB1249077F027B0563
:1050EF007A4D79CC1249077E077FD012498E7F0106
:1050FF007B057A4D79DD1249077F027B057A4D7961
:10510F00EE1249077E037FE812498E740190010C5D
:10511F00F0900116F090011AF07404A3F0900113AF
:10512F007406F0A374A4F09001097404F0A3749CA6
:10513F00F090011C7408F0A3E4F09001107403F0D8
:10514F00A374E8F0740F900117F07405A3F0743C8A
:10515F00A3F090010DF0A37405F0A37446F0E4FFE3
:10516F00FE900112F0124A33BE0102800302524731
:08517F00BF0002800302524749
:105187007401900115F0E4FE7F01124A33EF90019C
:105197000CF0E4FE7F02124A33EF900116F0E4FEB2
:1051A7007F03124A33EF90011AF0E4FE7F04124A9C
:1051B70033EF90011BF0E4FE7F05124A33EE9001B6
:1051C70013F0A3EFF0E4FE7F06124A33EE900109D5
:1051D700F0A3EFF0E4FE7F07124A33EE90011CF0D4
:1051E700A3EFF0E4FE7F08124A33EE900110F0A31C
:1051F700EFF0E4FE7F09124A33EF900117F0E4FE67
:105207007F0A124A33EF900118F0E4FE7F0B124A2F
:1052170033EF900119F0E4FE7F0C124A33EF90014F
:105227000DF0E4FE7F0D124A33EE90010EF0A3EF6E
:10523700F0E4FE7F0E124A33EF900112F002539C06
:105247007F017B057A4D79FF1249077F027B057A3B
:105257004E7910124907124AA3E4FE7F0A12498EBB
:10526700E4FEFF124AF6E4FDFEFF7C01124A051236
:105277004B19E4FEFF124A33BE0102800302536D4D
:08528700BF0002800302536D19
:10528F007401900115F0124AA3E4FE7F0A12498EB1
:10529F00E4FE7F0190010CE0FD7C00124A05E4FE64
:1052AF007F02900116E0FD7C00124A05E4FE7F03A9
:1052BF0090011AE0FD7C00124A05E4FE7F04900184
:1052CF001BE0FD7C00124A05E4FE7F05900113E010
:1052DF00FCA3E0FD124A05E4FE7F06900109E0FC05
:1052EF00A3E0FD124A05E4FE7F0790011CE0FCA33A
:1052FF00E0FD124A05E4FE7F08900110E0FCA3E0F8
:10530F00FD124A05E4FE7F09900117E0FD7C0012B3
:10531F004A05E4FE7F0A900118E0FD7C00124A0561
:10532F00E4FE7F0B900119E0FD7C00124A05E4FEBC
:10533F007F0C90010DE0FD7C00124A05E4FE7F0D0D
:10534F0090010EE0FCA3E0FD124A05E4FE7F0E90F3
:0E535F000112E0FD7C00124A05124B19802F4E
:10536D00E4900115F07F017B057A4E7921124907F2
:10537D007F027B057A4E79321249071249A6E4FE67
:10538D007FC812498E1249A67E027FBC12498E1229
:0B539D00798F30800C20810930000661
:1053A8001249A612347F900115E0B401028003026D
:0253B80055D0CE
:1053BA00900112E0B401005003025528E0B40A013A
:0653CA00D3400302552848
:1053D000E0FB24FFFFE434FFFEE4FC7D0A12014100
:1053E000EF2410FFE43E9001B9F0A3EFF0EB2400AE
:1053F000FBE43455FAC002C0039001B9E0FEA3E01B
:10540000FF124A33D005D0F0EEB5F002800302540B
:0A541000E0EFB5050280030254E04E
:10541A007F017B057A4E7943124907900112E0FB1E
:10542A00E4C0E0C0037B027A0179427D057C4E78B4
:10543A005412081D158115817F027B027A01794277
:10544A001249079001BAE02401FF9001B9E0340043
:10545A00FE124A33EF900106F09001BAE02402FFEF
:10546A009001B9E03400FE124A33EE9000FBF0A33B
:10547A00EFF09001BAE02403FF9001B9E03400FE96
:10548A00124A33EF9000FDF09001BAE02404FF9035
:10549A0001B9E03400FE124A33EE900102F0A3EFA4
:1054AA00F09001BAE02405FF9001B9E03400FE1241
:1054BA004A33EE900104F0A3EFF09001BAE024061B
:1054CA00FF9001B9E03400FE124A33EE900107F072
:0654DA00A3EFF00255D023
:1054E0007F017B057A4E79661249077F027B057A38
:1054F0004E7977124907E4900106F09000FB74039F
:10550000F0A374E8F07408A3F09001027403F0A310
:1055100074E8F0A37401F0A374F4F090010774052B
:08552000F0A37478F00255D0ED
:105528007F017B057A4E79661249077F027B057AEF
:105538004E7977124907E4FE7F10124A33BE555957
:03554800BF01564A
:10554B00E4FE7F11124A33EF900106F0E4FE7F1266
:10555B00124A33EE9000FBF0A3EFF0E4FE7F131240
:10556B004A33EF9000FDF0E4FE7F14124A33EE90C5
:10557B000102F0A3EFF0E4FE7F15124A33EE900127
:10558B0004F0A3EFF0E4FE7F16124A33EE9001070E
:06559B00F0A3EFF0802FE9
:1055A100E4900106F09000FB7403F0A374E8F0743A
:1055B10008A3F09001027403F0A374E8F0A374014E
:1055C100F0A374F4F09001077405F0A37478F090DF
:1055D1000106E0B40101D340067402900116F0E423
:1055E10090012EF0900132F0A3F090012FF0D2A99A
:1055F100127BE89000FEE4F0A3F00490010BF0C2EE
:105601000190015AF0E4FDFC90015DF0900109E088
:10561100FEA3E0FF121491C004C005C006C0077CC0
:105621006F7D127E837F3A12112C9001361200E3B6
:10563100E4FCFD90010EE0FEA3E0FF121491C00412
:10564100C005C006C0077C6F7D127E837F3A1211B0
:105651002C90013A1200E3E4FCFD90011CE0FEA352
:10566100E0FF121491C004C005C006C00774CDFC50
:1056710014FDFE743DFF12112C90013E1200E37ED9
:0C568100037FE812498E1249A6120003B4
:10568D001249B9EF900157F090015AE0B4050302A9
:10569D0062215014E014602014700302598324FE1B
:1056AD007003025BEE02798CE024F970030268A9A5
:0856BD0014700302775C80C841
:1056C500D2B2D2B3D2B4900157E0B40155300152F1
:0856D500900116E06403602758
:1056DD00740190010BF0740590015AF0127BE89063
:1056ED000119E0FBE4900130F0A3EBF0A3E4F0A38B
:0756FD00F090012FF08089FD
:1057040012497B7F017B057A4E79881249077F0213
:105714007B057A4E79991249071249A67E077FD0F4
:0A57240012498E900157E0B4020311
:0D572E00123344900157E0B4035330015092
:08573B00900116E064026022F7
:10574300740290015AF0127BE8900119E0FBE49097
:105753000130F0A3EBF0A3E4F0A3F090012FF002EB
:02576300798C3F
:1057650012497B7F017B057A4E79AA1249077F0290
:105775007B057A4E79991249071249A67E077FD093
:1057850012498E02568D7F05124C15EE900167F079
:0F579500A3EFF090010CE0B40102800302586111
:1057A400900106E0600F14600C14604214603F1412
:0557B400607502586160
:1057B900E4FCFD900167E0FEA3E0FF121491C00430
:1057C900C005C006C00790013E121285C004C0057D
:1057D900C006C0077455FEFCFD743FFF12112C1260
:1057E9001495EF9000FDF0806FE4FCFD900167E0F7
:1057F900FEA3E0FF121491C004C005C006C00790C3
:10580900013E121285C004C005C006C0077CDD7DBB
:10581900607E8A7F3E12112C121495EF9000FDF0E4
:105829008036E4FCFD900167E0FEA3E0FF121491CD
:10583900C004C005C006C00790013E121285C0040D
:10584900C005C006C007E4FEFCFD743FFF12112C21
:10585900121495EF9000FDF09000FBE0C0E0A3E08A
:10586900C0E0A3E0FBE4C0E0C0037B027A01794217
:105879007D057C4E78BB12081D74FC2581F581904D
:1058890000FDE070067441900148F07B027A0179CD
:1058990042900106E0FD127B947F017B027A017937
:1058A9004212490790011BE0FF124C15EE9001BB13
:1058B900F0A3EFF0E4FCFD900167E0FEA3E0FF1226
:1058C9001491C004C005C006C00790013E1212859C
:1058D900C004C005C006C0077466FEFCFD743FFF26
:0E58E900121522BFFF0280069000FDE070192C
:1058F7007B027A0179427D057C4E78CC12081D74B3
:0959070006900142F0C201806526
:10591000E4FCFD9001BBE0FEA3E0FF121491C00483
:10592000C005C006C00790013E121285C004C00524
:10593000C006C007E4FCFD900167E0FEA3E0FF1293
:105940001491C004C005C006C00790013E12128524
:10595000C004C005C006C0077B027A0179427D05FC
:105960007C4E78DD12081D74F82581F58174029053
:105970000142F0D2017F027B027A0179421249078B
:1059800002568DD2B3D2B41247C27F05124C15E431
:10599000FCFD121491C004C005C006C00790013E72
:1059A000121285C004C005C006C0077466FEFCFD67
:0959B000743FFF121522BFFF3EF7
:1059B900C201740890015AF0E4A3F07404A3F01230
:1059C90047C2127BE87F05124C15EE900126F0A321
:1059D900EFF090011BE0FF124C15EE90012AF0A3A5
:1059E900EFF0900130E4F0A37404F002568D9001B9
:0559F90057E0B402506C
:1059FE007B057A4E79EE127ABFEF6401600302796D
:015A0E008C0B
:105A0F007F05124C15EE900126F0A3EFF01247C25E
:105A1F001249A6740890015AF0E4A3F07402A3F09F
:105A2F00127BE890011BE0FF124C15EE90012AF05B
:105A3F00A3EFF0900130E4F0A37404F002568D7BD5
:105A4F00027A0179427D057C4E78FF12081D7B0298
:105A5F007A01794D900106E0FD127B947406900156
:105A6F0042F07F017B027A0179421249079001309F
:105A7F00E0C0E0A3E0C0E07B027A0179427D057CC3
:105A8F004F781012081D158115817402900142F094
:075A9F0090012DE0B4010AA3
:0A5AA6007407900143F0C2B28002C1
:105AB000D2B27F027B027A0179421249079001300B
:0D5AC000E06003025BE0A3E06003025BE036
:105ACD00C2B275FD0175ED0175DD42D2DE90013A70
:105ADD0012009CE4FCFD900104E0FEA3E0FF121413
:105AED009112112C121495EE900161F0A3EFF0902C
:105AFD0000FEE4F0A3F0C0E0C0E07461C0E07445C6
:105B0D00C0E0900102E0FEA3E0FFE4FCFD12149161
:105B1D00121288C004C005C006C007E4FCFD74C89D
:105B2D00FE7442FF12112C121495EE900100F0A399
:105B3D00EFF07B027A0179427D057C4F78211208C6
:105B4D001D7406900142F07F017B027A01794212A9
:105B5D0049077F027B057A4F79321249077F01127F
:105B6D0048DC900161E0FEA3E0FF7D031240EFEE03
:105B7D0090015FF0A3EFF07F027B057A4F7932122F
:105B8D004907E4FF1248DC740490015AF0E49001D7
:065B9D005DF0900156F0DE
:105BA30090015FE0FCA3E0FD900156E0FA2AFB249C
:105BB3007DF582E43401F583ECF0A3EDF090016709
:105BC300E0FCA3E0FDEB2491F582E43401F583ECE2
:105BD300F0A3EDF0900156E004F0B40AC390013253
:105BE300E4F0A3F090012FF002568DC2B29001575A
:105BF300E064016004E0B40306740590015DF09075
:095C03000100E0705DA3E070599E
:105C0C009000FFE004F09000FE7003E004F0E4C0AC
:105C1C00E0C0E07461C0E07445C0E0E4FCFD9001BC
:105C2C005FE0FEA3E0FF121491C004C005C006C0E3
:105C3C000790013A121285121288C004C005C006E2
:105C4C00C007E4FCFD74C8FE7442FF12112C121440
:105C5C0095EE900100F0A3EFF0900157E0B4026DC7
:105C6C007B057A4E79EE127ABFEF640160030279FC
:015C7C008C9B
:105C7D007F05124C15EE900126F0A3EFF01247C2EE
:105C8D001249A6740890015AF0E4A3F07402A3F02F
:105C9D009000FEE0FAA3E0FB900122EAF0A3EBF006
:105CAD00900132E0FAA3E0FB900124EAF0A3EBF0BF
:105CBD0090011BE0FF124C15EE90012AF0A3EFF0BE
:105CCD00900130E4F0A37404F002568D90012FE0A2
:0D5CDD00F5F0900158E065F07003025E9C48
:105CEA0090015DE0B40001D34003E014F090011B81
:105CFA00E0FF124C15EE9001BBF0A3EFF07F041207
:105D0A000771EE90018DF0A3EFF09001BD1200EF44
:095D1A0000000000E4900156F0C5
:105D2300900156E025E0247FF582E43401F583E019
:105D3300FCA3E0FD900156E0FA2AFF247DF582E4FE
:105D43003401F583ECF0A3EDF09001BD12009CEF5C
:105D5300247DF582E43401F583E0FEA3E0FFE4FC57
:105D6300FD12012C9001BD1200E3900156E004F0F6
:105D7300B408AD75F0039001BD1200D7120117905E
:105D8300015FEEF0A3EFF0A3E0FEA3E0FFE4FCFD70
:105D9300121491C004C005C006C00774CDFC14FDE5
:105DA300FE743CFF12112C121495EE900175F0A3B2
:105DB300EFF090015FE0FCA3E0FDA3E0FAA3E0FBBA
:105DC300900176E0F8EBC398FB900175E0F8EA9850
:105DD300FAF5F0ECB5F004EDB50300401EE0FAA3CC
:105DE300E0FB900162E02BFB900161E03AFAF5F0F1
:0B5DF300ECB5F005EDB50301D3401541
:105DFE00900161E0FEA3E0FF7D041240EFEE900102
:105E0E005FF0A3EFF01207B1EE9001A1F0A3EFF057
:0F5E1E009001BD1200EF00000000E4900156F06B
:105E2D00900156E025E02493F582E43401F583E0FA
:105E3D00FCA3E0FD900156E0FA2AFF2491F582E4DF
:105E4D003401F583ECF0A3EDF09001BD12009CEF51
:105E5D002491F582E43401F583E0FEA3E0FFE4FC38
:105E6D00FD12012C9001BD1200E3900156E004F0EB
:105E7D00B408AD75F0039001BD1200D71201179053
:105E8D000167EEF0A3EFF090012FE0900158F09034
:105E9D000167E0B40006A3E0B40001D35003025F34
:105EAD00A1E4FCFD900167E0FEA3E0FF121491C098
:105EBD0004C005C006C00790013E121285C004C083
:105ECD0005C006C0079000FDE0FB7A00E433E45006
:105EDD000114FCFDAE02AF03121454C004C005C082
:105EED0006C007E4FCFD900110E0FEA3E0FF1214D4
:105EFD0091C004C005C006C0077C6F7D127E837FF4
:105F0D003A12112C12112C121522BFFF028003021E
:025F1D005FA182
:105F1F00900167E0FAA3E0FB900126EAF0A3EBF013
:105F2F001247C29000FEE0FAA3E0FB900122EAF0D4
:105F3F00A3EBF0900132E0FAA3E0FB900124EAF02A
:105F4F00A3EBF090011BE0FF124C15EE90012AF02D
:0A5F5F00A3EFF0900116E0B4011D5D
:105F690090010DE0FBE4900130F0A3EBF074059093
:0D5F7900015AF0900132E4F0A3F002798C9F
:105F86001249A6740890015AF0E4A3F004A3F09015
:105F96000130E4F0A37404F002568DE4FCFD900198
:105FA60067E0FEA3E0FF121491C004C005C006C05E
:105FB6000790013E121285C004C005C006C00774D2
:0D5FC60066FEFCFD743FFF121522BFFF5F59
:105FD3001247C21249A6740890015AF0E4A3F07460
:105FE30004A3F09000FEE0FAA3E0FB900122EAF0A4
:105FF300A3EBF0900132E0FAA3E0FB900124EAF076
:10600300A3EBF0900167E0FAA3E0FB900126EAF02E
:10601300A3EBF090011BE0FF124C15EE90012AF068
:10602300A3EFF0900130E4F0A37404F002568D90D6
:1060330000FEE0FAA3E0F4FBEAF4FA0BEB70010ACA
:10604300C002C0037B027A0179427D057C4F78430D
:1060530012081D1581158190010BE06401600A90FF
:096063000106E0B40101D3401074
:10606C007B027A017944900106E0FD127B94801743
:10607C007444900145F014A3F0743AA3F090010B12
:10608C00E02430900148F090012CE0FA7404C39A9B
:10609C00900142F07406A3F07F017B027A017942F1
:0C60AC0012490790015DE060030261BD35
:1060B800900132E06003026141A3E0707C90012FFF
:1060C800E0FBE4C0E0C003FCFD90015FE0FEA3E05C
:1060D800FF121491C004C005C006C00790013A120F
:1060E8001285C004C005C006C0077C6F7D127E8380
:1060F8007F3A12112CC004C005C006C007E4FCFD9D
:10610800900167E0FEA3E0FF121491C004C005C02F
:1061180006C00790013E121285C004C005C006C023
:10612800077B027A0179427D057C4F785412081D5D
:1061380074F62581F581026213900132E0C0E0A374
:10614800E0C0E0E4FCFD90015FE0FEA3E0FF121474
:1061580091C004C005C006C00790013A121285C05C
:1061680004C005C006C0077C6F7D127E837F3A128B
:10617800112CC004C005C006C007E4FCFD900167EF
:10618800E0FEA3E0FF121491C004C005C006C007DA
:1061980090013E121285C004C005C006C0077B02EC
:1061A8007A0179427D057C4F786712081D74F625BF
:0561B80081F581805615
:1061BD00E5FDFF7E00E4FC7D64120141E4FC7DFF02
:1061CD00120155C006C007E4FCFD9001BBE0FEA323
:1061DD00E0FF121491C004C005C006C00790013E37
:1061ED00121285C004C005C006C0077B027A017972
:1061FD00427D057C4F787A12081D74FA2581F58150
:10620D007425900151F07F027B027A017942124987
:10621D000702568DD2B2D2B41247C27F05124C1569
:10622D00E4FCFD121491C004C005C006C007900126
:10623D003E121285C004C005C006C0077466FEFC80
:0A624D00FD743FFF121522BFFF4150
:106257001247C21249A6C201740890015AF0E4A37A
:10626700F07404A3F0900167E0FAA3E0FB90012625
:10627700EAF0A3EBF090011BE0FF124C15EE900142
:106287002AF0A3EFF0900130E4F0A37404F0025673
:086297008D900157E0B4024DA7
:10629F007B057A4F798C127ABFEF64016003027924
:0162AF008C62
:1062B0007F05124C15EE900126F0A3EFF090011B24
:1062C000E0FF124C15EE90012AF0A3EFF01247C246
:1062D0001249A6740890015AF0E4A3F07402A3F0E6
:1062E000900130E4F0A37404F002568D7B027A0131
:1062F00079427D057C4F789D12081D7B027A0179D9
:106300004A900106E0FD127B947406900142F07FF2
:10631000017B027A017942124907900130E0C0E026
:10632000A3E0C0E07B027A0179427D057C4F7810C2
:1063300012081D158115817402900142F090012D03
:04634000E0B4010ABA
:0A6344007407900143F0C2B3800219
:10634E00D2B37F027B027A01794212490790013063
:0D635E00E0600302689BA3E0600302689BFF
:10636B0090013612009CE4FCFD74A0FE7441FF12F8
:10637B00112C121495EE90016BF0A3EFF0E4FCFDE1
:10638B00900113E0FEA3E0FF121491C004C005C0FE
:10639B0006C0077C6F7D127E837F3A12112CC004DE
:1063AB00C005C006C0079000FDE0FF7E00E433E4AB
:1063BB00500114FCFD12145412112CC004C005C062
:1063CB0006C00790013E121129121495EE90016F31
:1063DB00F0A3EFF0900106E0705D900117E0FF7EF7
:1063EB0000E433E4500114FCFD121454C004C00546
:1063FB00C006C0077C6F7D127E837F3A12112CC0C2
:10640B0004C005C006C0079000FDE0FDFFE4FE33AD
:10641B00E4500114FDFC12145412112CC004C005DD
:10642B00C006C00790013E121129121495EE90017F
:10643B0071F0A3EFF08064900118E0FBE433E450BB
:10644B000114FCFD7E00AF03121454C004C005C040
:10645B0006C0077C6F7D127E837F3A12112CC0041D
:10646B00C005C006C0079000FDE0FD7C00E4C0E065
:10647B00EDFFD0E0FE33E4500114FDFC1214541276
:10648B00112CC004C005C006C00790013E12112993
:10649B00121495EE900171F0A3EFF0900107E0FE5E
:1064AB00A3E0FFE4FCFD121491C004C005C006C0BC
:1064BB00077C6F7D127E837F3A12112CC004C005BE
:1064CB00C006C0079000FDE0FD7C00E4C0E0EDFFDE
:1064DB00D0E0FE33E4500114FDFC12145412112CC5
:1064EB00C004C005C006C00790013E12112912144A
:1064FB0095EE900165F0A3EFF09000FBE0FEA3E0BA
:10650B00FF900102E0FCA3E0FD12017DE4FCFD1213
:10651B001491C004C005C006C007749AFC14FDFE9C
:10652B00743FFF12112CC004C005C006C007E4FC69
:10653B00FD7461FE7445FF12112C121495EE90013F
:10654B0034F0A3EFF09000FDE0FF7E00E433E45065
:10655B000114FCFD121454C004C005C006C007741E
:10656B0066FCFD74B6FE743FFF12112CC004C0050F
:10657B00C006C00790013E121129121495EE90012E
:10658B0073F0A3EFF090013E12009CE4FEFCFD744F
:10659B003FFF12112C121495EE900177F0A3EFF040
:1065AB0090011BE0B4046DE4FCFD900107E0FEA339
:1065BB00E0FF121491C004C005C006C0077C6F7DBC
:1065CB00127E837F3A12112CC004C005C006C0078F
:1065DB009000FDE0FF7E00E433E4500114FCFD125B
:1065EB00145412112CC004C005C006C007E4FCFDF6
:1065FB007480FE743FFF120FD5C004C005C006C0E7
:10660B000790013E121129121495EE900169F0A327
:10661B00EFF0801D90013E12009CE4FCFD7428FEFF
:10662B007441FF12112C121495EE900169F0A3EF37
:10663B00F090013E12009C900118E0FF7E00E433C5
:10664B00E4500114FCFD12145412112C121495EE8B
:10665B0090017BF0A3EFF0900106E0FA6402600377
:10666B00BA032D90013612009C9000FDE0FF7E00D6
:10667B00E4FC7D32120141EE33E4500114FDFC12B7
:10668B00145412112C121495EE90016DF0A3EFF02F
:10669B00900106E0B4043A9000FBE4FCFDE0FEA39D
:1066AB00E0FF121491C004C005C006C0077C297D11
:1066BB005C7E8F7F3D12112CC004C005C006C00745
:1066CB00900136121129121495EE90016DF0A3EF83
:1066DB00F0900106E0B40101D3404BE4FCFD9001C6
:0266EB006DE060
:1066ED00FEA3E0FF121491C004C005C006C00790C0
:1066FD00013612009CE4FCFD7448FE7442FF121139
:10670D002C121522BFFF1D90013612009CE4FCFDDA
:10671D007448FE7442FF12112C121495EE90016D07
:10672D00F0A3EFF0900106E0B40101D3400674012F
:10673D0090010BF0C202E4900159F090015BF090D2
:10674D000167E0FAA3E0FB900163EAF0A3EBF0E44C
:10675D0090015DF0900179F0A3F090015EF0900052
:10676D00FEF0A3F0C0E0C0E07461C0E07445C0E08D
:10677D00900102E0FAA3E0FBE4FCFDAE02AF0312D0
:10678D001491121288C004C005C006C007E4FCFDB8
:10679D0074C8FE7442FF12112C121495EE90010074
:1067AD00F0A3EFF0C2B375FE0175EE0175DE42D2B6
:1067BD00DEC20390013612009CE4FCFD900102E064
:1067CD00FEA3E0FF12149112112C121495EE9001FC
:1067DD0061F0A3EFF07B027A0179427D057C4F7861
:1067ED00AF12081D7406900142F07F017B027A0101
:1067FD0079421249077F027B057A4F793212490798
:10680D007F011248DC900161E0FEA3E0FF7D0612DE
:10681D0040EFEE90015FF0A3EFF07F027B057A4F22
:0F682D007932124907E4FF1248DCE4900156F07B
:10683C0090015FE0FCA3E0FD900156E0FA2AFB24F6
:10684C007DF582E43401F583ECF0A3EDF090016763
:10685C00E0FCA3E0FDEB2491F582E43401F583EC3C
:10686C00F0A3EDF090011BE0FF124C15900156E0E7
:10687C00FA2A24A5F582E43401F583EEF0A3EFF0B7
:10688C00900156E004F0B40AA7740790015AF090F6
:10689C000132E4F0A3F090012FF002568DC2B390B8
:1068AC000157E064016004E0B40306740590015DD7
:0B68BC00F0900100E0705DA3E0705957
:1068C7009000FFE004F09000FE7003E004F0E4C0E5
:1068D700E0C0E07461C0E07445C0E0E4FCFD9001F5
:1068E7005FE0FEA3E0FF121491C004C005C006C01C
:1068F70007900136121285121288C004C005C0061F
:10690700C007E4FCFD74C8FE7442FF12112C121478
:1069170095EE900100F0A3EFF0900134E0706EA3C4
:03692700E0706AB3
:10692A001247C21249A6740890015AF0E4A3F0A3D0
:10693A00F09000FEE0FAA3E0FB90011EEAF0A3EB60
:10694A00F0900132E0FAA3E0FB900120EAF0A3EB19
:10695A00F0900167E0FAA3E0FB900126EAF0A3EBCE
:10696A00F0900179E0FAA3E0FB900128EAF0A3EBAA
:10697A00F090011BE0FF124C15EE90012AF0A3EFF4
:10698A00F0900130E4F0A37404F0900157E0B402EF
:06699A00028003026A23E3
:0E69A0007B057A4F798C127ABFEF6401707517
:1069AE001247C21249A6740190010BF074089001AF
:1069BE005AF0E4A3F07402A3F09000FEE0FAA3E014
:1069CE00FB90011EEAF0A3EBF0900132E0FAA3E097
:1069DE00FB900120EAF0A3EBF0900167E0FAA3E050
:1069EE00FB900126EAF0A3EBF0900179E0FAA3E028
:1069FE00FB900128EAF0A3EBF090011BE0FF124C94
:106A0E0015EE90012AF0A3EFF0900130E4F0A3749C
:0B6A1E0004F002568D300303026BDF12
:106A290090012FE0F5F0900158E065F07003026DD8
:016A3900BBA1
:106A3A0090015DE0B40001D34003E014F07F071237
:106A4A000771EE90018DF0A3EFF09001BD1200EFF7
:096A5A0000000000E4900156F078
:106A6300900156E025E0247FF582E43401F583E0CC
:106A7300FCA3E0FD900156E0FA2AFF247DF582E4B1
:106A83003401F583ECF0A3EDF09001BD12009CEF0F
:106A9300247DF582E43401F583E0FEA3E0FFE4FC0A
:106AA300FD12012C9001BD1200E3900156E004F0A9
:106AB300B408AD75F0039001BD1200D71201179011
:106AC300015FEEF0A3EFF0A3E0FEA3E0FFE4FCFD23
:106AD300121491C004C005C006C00774CDFC14FD98
:106AE300FE743CFF12112C121495EE900175F0A365
:106AF300EFF090015FE0FCA3E0FDA3E0FAA3E0FB6D
:106B0300900176E0F8EBC398FB900175E0F8EA9802
:106B1300FAF5F0ECB5F004EDB50300401EE0FAA37E
:106B2300E0FB900162E02BFB900161E03AFAF5F0A3
:0B6B3300ECB5F005EDB50301D34015F3
:106B3E00900161E0FEA3E0FF7D071240EFEE9001B1
:106B4E005FF0A3EFF01207B1EE9001A1F0A3EFF00A
:0F6B5E009001BD1200EF00000000E4900156F01E
:106B6D00900156E025E02493F582E43401F583E0AD
:106B7D00FCA3E0FD900156E0FA2AFF2491F582E492
:106B8D003401F583ECF0A3EDF09001BD12009CEF04
:106B9D002491F582E43401F583E0FEA3E0FFE4FCEB
:106BAD00FD12012C9001BD1200E3900156E004F09E
:106BBD00B408AD75F0039001BD1200D71201179006
:106BCD000167EEF0A3EFF090012FE0900158F00275
:026BDD006DBB8E
:106BDF0090012FE0F5F0900158E065F07003026D21
:016BEF00BBEA
:106BF00090015DE0B40001D34003E014F01207B14E
:106C0000EE9001A1F0A3EFF09001BD1200EF0000A3
:076C10000000E4900156F0C2
:106C1700900156E025E02493F582E43401F583E002
:106C2700FEA3E0FF900156E0FA2AFD7C002491F5CF
:106C370082E43401F583EEF0A3EFF09001BD12007A
:106C47009CED2491F582E43401F583E0FEA3E0FF97
:106C5700E4FD12012C9001BD1200E3900156E004FF
:106C6700F0B408AC75F0039001BD1200D7120117FC
:106C7700900167EEF0A3EFF0900106E0B4042FE473
:106C8700FCFD900165E0FEA3E0FF121491C004C073
:106C970005C006C00774CDFC14FDFE743CFF12113D
:106CA7002C121495EE900175F0A3EFF0801C900163
:106CB7003E12009C7C0A7DD77EA37F3B12112C12CB
:106CC7001495EE900175F0A3EFF0900167E0FCA337
:106CD700E0FD900165E0FAA3E0FB900176E0F8EBB8
:106CE700C398FB900175E0F8EA98FAF5F0ECB5F077
:106CF70004EDB50300401EE0FAA3E0FB900166E057
:106D07002BFB900165E03AFAF5F0ECB5F005EDB52F
:056D17000301D340134D
:106D1C00900165E0FEA3E0FF1245ABEE900167F039
:106D2C00A3EFF07F07120771EE90018DF0A3EFF047
:0F6D3C009001BD1200EF00000000E4900156F03E
:106D4B00900156E025E0247FF582E43401F583E0E1
:106D5B00FEA3E0FF900156E0FA2AFD7C00247DF5AE
:106D6B0082E43401F583EEF0A3EFF09001BD120045
:106D7B009CED247DF582E43401F583E0FEA3E0FF76
:106D8B00E4FD12012C9001BD1200E3900156E004CA
:106D9B00F0B408AC75F0039001BD1200D7120117C7
:106DAB0090015FEEF0A3EFF090012FE0900158F00F
:106DBB00900106E06009E0B401028003026E689066
:106DCB00016BE0FAF5F0A3E0FB90015FE0B5F00694
:0B6DDB00A3E0B50301D34003026E6883
:106DE6007F05124C15EE900126F0A3EFF01247C274
:106DF60075FD7F75ED7F75DD42D2DE1249A6740101
:106E060090010BF0C201740890015AF0E4A3F074EB
:106E160004A3F09000FEE0FAA3E0FB90011EEAF066
:106E2600A3EBF0900132E0FAA3E0FB900120EAF038
:106E3600A3EBF0900179E0FAA3E0FB900128EAF0D9
:106E4600A3EBF090011BE0FF124C15EE90012AF027
:106E5600A3EFF0900130E4F0A37404F01247C202ED
:106E6600568D900106E0FAB40101D35003026F3E3D
:106E760090016BE0FCA3E0FD90015FE0B50406A382
:106E8600E0B50501D34003026F3E900167E0FEA323
:106E9600E0FF900177E0FCA3E0FD900166E02DFDA8
:106EA600900165E03CFCF5F0EEB5F005EFB50501A7
:066EB600D35003026F3E01
:106EBC007F05124C15EE900126F0A3EFF01247C29D
:106ECC0075FD7F75ED7F75DD42D2DE1249A674012A
:106EDC0090010BF0C201740890015AF0E4A3F07415
:106EEC0004A3F09000FEE0FAA3E0FB90011EEAF090
:106EFC00A3EBF0900132E0FAA3E0FB900120EAF062
:106F0C00A3EBF0900179E0FAA3E0FB900128EAF002
:106F1C00A3EBF090011BE0FF124C15EE90012AF050
:106F2C00A3EFF0900130E4F0A37404F01247C20216
:106F3C00568D900106E06009E0B401028003026FF7
:016F4C00E064
:106F4D0090016FE0FAA3E0FB900167E0B50206A3A4
:076F5D00E0B50301D340770A
:0C6F6400900159E004F0B40301D3407028
:106F70007F05124C15EE900126F0A3EFF01247C2E8
:106F80001249A6740890015AF0E4A3F07403A3F028
:106F90009000FEE0FAA3E0FB90011EEAF0A3EBF004
:106FA000900132E0FAA3E0FB900120EAF0A3EBF0BD
:106FB000900179E0FAA3E0FB900128EAF0A3EBF05E
:106FC00090011BE0FF124C15EE90012AF0A3EFF0A8
:0B6FD000900130E4F0A37404F0800591
:106FDB00E4900159F0900106E06009E0B4010280F1
:106FEB0003027195900173E0FAA3E0FB900167E057
:0E6FFB00B50206A3E0B50301D3500302719561
:10700900900179E0FAA3E0FB900167E0B50206A3DD
:07701900E0B50301D3401EA6
:10702000900167E0FAA3E0FB900179EAF0A3EBF0AE
:0E703000900106E06003027195C202027195A4
:10703E00900172E0FB900171E0C313CB13CBFA9079
:10704E000179E0FCA3E0FD900168E0F8EDC398FD46
:10705E00900167E0F8EC98B50205EDB50301D34059
:10706E0002D202900171E0FCA3E0FD900179E0FAFA
:10707E00A3E0FB900168E0F8EBC398FB900167E09A
:10708E00F8EA98B50405EBB50501D35003027195E6
:0D709E0090010BE0B40101D3500302712BEF
:1070AB00E014F0740290015AF01247C2900122E4EE
:1070BB00F0A3F0A3F0A3F09000FEE0FAA3E0FB90A6
:1070CB00011EEAF0A3EBF0900132E0FAA3E0FB9093
:1070DB000120EAF0A3EBF0900167E0FAA3E0FB904C
:1070EB000126EAF0A3EBF0900179E0FAA3E0FB9024
:1070FB000128EAF0A3EBF090011BE0FF124C15EE18
:10710B0090012AF0A3EFF090010DE0FBE490013029
:10711B00F0A3EBF0A3E4F0A3F090012FF002568D57
:10712B001247C21249A6740890015AF0E4A3F0A3C7
:10713B00F09000FEE0FAA3E0FB90011EEAF0A3EB57
:10714B00F0900132E0FAA3E0FB900120EAF0A3EB10
:10715B00F0900167E0FAA3E0FB900126EAF0A3EBC5
:10716B00F0900179E0FAA3E0FB900128EAF0A3EBA1
:10717B00F090011BE0FF124C15EE90012AF0A3EFEB
:10718B00F0900130E4F0A37404F0900106E0FAB43F
:10719B0001028003027339900173E0FCF5F0A3E068
:1071AB00FD900167E0B5F006A3E0B50501D35003F0
:0371BB0002733923
:1071BE00900130E06003027339A3E060030273397B
:1071CE0090017BE0C0E0A3E0C0E0900163E0FAA391
:1071DE00E0FB900168E0F8EBC398FF900167E0F8E0
:1071EE00EA98FE120212D003D0F0EEB5F004EFB51D
:0771FE0003004003027319B6
:1072050090015BE004F0B40101D34002D202900189
:0B7215005BE0B40401D35003027320BF
:0D72200090010BE0B40101D350030272ADE8
:10722D00E014F0740290015AF01247C2900122E46A
:10723D00F0A3F0A3F0A3F09000FEE0FAA3E0FB9022
:10724D00011EEAF0A3EBF0900132E0FAA3E0FB900F
:10725D000120EAF0A3EBF0900167E0FAA3E0FB90C8
:10726D000126EAF0A3EBF0900179E0FAA3E0FB90A0
:10727D000128EAF0A3EBF090011BE0FF124C15EE94
:10728D0090012AF0A3EFF090010DE0FBE4900130A6
:10729D00F0A3EBF0A3E4F0A3F090012FF002568DD4
:1072AD001247C21249A6740890015AF0E4A3F0A344
:1072BD00F09000FEE0FAA3E0FB90011EEAF0A3EBD4
:1072CD00F0900132E0FAA3E0FB900120EAF0A3EB8D
:1072DD00F0900167E0FAA3E0FB900126EAF0A3EB42
:1072ED00F0900179E0FAA3E0FB900128EAF0A3EB1E
:1072FD00F090011BE0FF124C15EE90012AF0A3EF68
:0C730D00F0900130E4F0A37404F080075D
:10731900C202E490015BF0900130E4F0A3743CF008
:10732900900167E0FAA3E0FB900163EAF0A3EBF0B8
:0D733900900106E0B40101D350030274433B
:10734600900165E0FAA3E0FBA3E0B50205A3E0B572
:07735600030040182003159D
:10735D00D202D203900135E02410FB900134E034C9
:10736D000EF0A3EBF090016DE0FAA3E0FB90015F4E
:10737D00E0B50205A3E0B50300400302744320030A
:10738D000302744390016BE0FAA3E0FB90015FE010
:10739D00B50206A3E0B50301D35003027443900177
:1073AD0067E0FCA3E0FD900177E0FAA3E0FB90011C
:1073BD0066E02BFB900165E03AFAF5F0ECB5F004D0
:0673CD00EDB50300507055
:1073D300740190010BF01247C21249A67408900180
:1073E3005AF0E4A3F0A3F09000FEE0FAA3E0FB90D0
:1073F300011EEAF0A3EBF0900132E0FAA3E0FB9068
:107403000120EAF0A3EBF0900167E0FAA3E0FB9020
:107413000126EAF0A3EBF0900179E0FAA3E0FB90F8
:107423000128EAF0A3EBF090011BE0FF124C15EEEC
:1074330090012AF0A3EFF0900130E4F0A37404F07C
:107443009001BD1200EF0000000090011BE0FF124D
:0F7453004C15EE9001B5F0A3EFF0E4900156F068
:10746200900156E025E024A7F582E43401F583E09B
:10747200FEA3E0FF900156E0FA2AFD7C0024A5F568
:1074820082E43401F583EEF0A3EFF09001BD120027
:107492009CED24A5F582E43401F583E0FEA3E0FF30
:1074A200E4FD12012C9001BD1200E3900156E004AC
:1074B200F0B408AC75F0039001BD1200D7120117A9
:1074C2009001BBEEF0A3EFF0900169E0F5F0A3E0CC
:1074D200FB9001BBE0B5F005A3E0B5030040030259
:0274E2007564CF
:0C74E40090015EE004F0B40301D3407995
:1074F0001247C21249A6740190010BF07408900162
:107500005AF0E4A3F07405A3F0900130E4F0A37402
:1075100004F09000FEE0FAA3E0FB90011EEAF0A365
:10752000EBF0900132E0FAA3E0FB900120EAF0A337
:10753000EBF0900167E0FAA3E0FB900126EAF0A3EC
:10754000EBF0900179E0FAA3E0FB900128EAF0A3C8
:10755000EBF09001BBE0FAA3E0FB90012AEAF0A374
:04756000EBF08005C7
:10756400E490015EF09000FEE0C0E0A3E0C0E07BA8
:10757400027A0179427D057C4F784312081D1581FA
:10758400158190010BE06401600A900106E0B401EA
:0475940001D34010CF
:107598007B027A017944900106E0FD127B94801702
:1075A8007443900145F004A3F0743AA3F090010BE2
:0A75B800E02430900148F020020AA0
:0A75C20090012CE0900142F0800DD2
:1075CC0090012DE0B401067404900142F074059012
:1075DC000143F07F017B027A017942124907900145
:0775EC005DE060030276F888
:1075F300900132E0600302767CA3E0707C90012F5F
:10760300E0FBE4C0E0C003FCFD90015FE0FEA3E00B
:10761300FF121491C004C005C006C00790013612C2
:107623001285C004C005C006C0077C6F7D127E832F
:107633007F3A12112CC004C005C006C007E4FCFD4C
:10764300900167E0FEA3E0FF121491C004C005C0DF
:1076530006C00790013E121285C004C005C006C0D3
:10766300077B027A0179427D057C4F785412081D0D
:1076730074F62581F58102774E900132E0C0E0A3D4
:10768300E0C0E0E4FCFD90015FE0FEA3E0FF121424
:1076930091C004C005C006C007900136121285C010
:1076A30004C005C006C0077C6F7D127E837F3A123B
:1076B300112CC004C005C006C007E4FCFD9001679F
:1076C300E0FEA3E0FF121491C004C005C006C0078A
:1076D30090013E121285C004C005C006C0077B029C
:1076E3007A0179427D057C4F786712081D74F6256F
:0576F30081F5818056C5
:1076F800E5FEFF7E00E4FC7D64120141E4FC7DFFB1
:10770800120155C006C007E4FCFD9001BBE0FEA3D2
:10771800E0FF121491C004C005C006C00790013EE6
:10772800121285C004C005C006C0077B027A017921
:10773800427D057C4F787A12081D74FA2581F581FF
:107748007425900151F07F027B027A017942124937
:107758000702568DD2B2D2B390015CE0B403028026
:1077680050500BE06012146022146032807AE024DA
:08777800FC6051146061807097
:107780007B027A0179427D057C4F78C012081DD2B8
:10779000B4805D7B027A0179427D057C4F78D112FD
:1077A000081DD2B4804A7B027A0179427D057C4F64
:1077B00078E212081DC2B480377B027A0179427DDB
:1077C000057C4F78F312081DC2B480247B027A0135
:1077D00079427D057C50780412081DC2B480117B6B
:1077E000027A0179427D057C50781512081DC2B4D9
:1077F0007406900142F07F017B027A0179421249BE
:0B78000007900130E0701EA3E0701A3A
:10780B00124957900130E4F0A37404F090015BE04F
:10781B0004F0B40501D34002E4F090015BE0B40343
:10782B00030278B9500CE0601A14604214605F02D6
:10783B007971E024FC70030278D914700302793853
:03784B000279714E
:10784E00900123E0F4FB900122E0F4FA0BEB7001BF
:10785E000AC002C0037B027A0179427D057C507812
:10786E002612081D15811581027971900124E0C040
:10787E00E0A3E0C0E07B027A0179427D057C50787E
:10788E003712081D1581158102797190011EE0C015
:10789E00E0A3E0C0E07B027A0179427D057C50785E
:1078AE004812081D15811581027971900120E0C0E2
:1078BE00E0A3E0C0E07B027A0179427D057C50783E
:1078CE005912081D15811581027971E4FCFD900194
:1078DE0026E0FEA3E0FF121491C004C005C006C04E
:1078EE000790013E121285C004C005C006C007E411
:1078FE00FCFD900128E0FEA3E0FF121491C004C02D
:10790E0005C006C00790013E121285C004C005C016
:10791E0006C0077B027A0179427D057C50786A1297
:10792E00081D74F82581F5818039E4FCFD90012A4B
:10793E00E0FEA3E0FF121491C004C005C006C0070C
:10794E0090013E121285C004C005C006C0077B021E
:10795E007A0179427D057C50787C12081D74FC25D5
:10796E0081F5817F027B027A0179421249079001EB
:05797E0057E0B402090E
:0C798300120003740190015AF002568DAE
:10798F00900116E0B401004007E0B40301D34006B4
:10799F007401900116F090011BE0B40401D3400371
:1079AF007404F0900113E0FAA3E0FBBA0603B440AD
:1079BF00004009BA0704BB6C01D3400A900113744D
:1079CF0006F0A374A4F0900109E0FAA3E0FBBA0358
:1079DF0003B4E8004009BA0704BBD001D3400A90B2
:1079EF0001097404F0A3749CF090011CE0FAA3E069
:1079FF00FBBA0703B4D0004009BA0B04BBB801D3DC
:107A0F00400990011C7408F0A3E4F0900110E0FA13
:107A1F00A3E0FBBA0103B4F4004009BA0404BBB0FD
:107A2F0001D3400A9001107403F0A374E8F09001A1
:107A3F0017E0B405004007E0B41901D34006740FF6
:107A4F00900117F0900118E0B403004007E0B40A6A
:107A5F0001D340067405900118F0900119E0B41E8F
:107A6F0000400AE0FB7A00B4F001D34006743C906A
:107A7F000119F090010DE0B41E00400AE0FB7A00FE
:107A8F00B4F001D34006743C90010DF090010EE06C
:107A9F00FAA3E0FBBA0303B4E8004009BA0704BB3A
:107AAF00D001D3400A90010E7405F0A37446F02262
:107ABF008B2F8A30893112000374199001D5F09001
:107ACF00012DE024FF92057F01AB2FAA30A93112BF
:107ADF0049077B027A0179C17D057C50788E1208A7
:107AEF001D74069001C3F0E49001D6F0A3F090014D
:067AFF00D7E0640260758F
:107B05001249B9EF9001D7F064016004E0B403298C
:077B15009001D6E0B401105D
:107B1C00E4F074069001C3F074209001CAF0801256
:107B2C0074019001D6F074209001C3F0740690019A
:107B3C00CAF07F027B027A0179C112490790012DAC
:107B4C00E0B4010874079001D0F080067420900115
:0E7B5C00D0F0A205E433FA90012DE06A6093A8
:107B6A00E024FF92059001D5E014F07086E4FF222C
:067B7A009001D6E0FF229D
:107B80004E6943444E694D484C69506F4C694F4EA5
:047B9000534C4120F1
:0D7B94008B218A2289238D07E49001D8F00F
:0A7BA1009001D8E0B40216BF0313F0
:107BAB00AB21AA22A923744912002A0523E52370CD
:107BBB00020522EF25E025E0FE9001D8E02E907B18
:107BCB008093AD21AC22A82312000E0523E5237070
:0D7BDB000205229001D8E004F0B404BA22A3
:107BE80090011EE4F0A3F0A3F0A3F0A3F0A3F0A388
:107BF800F0A3F0A3F0A3F0A3F0A3F0A3F0A3F02266
:00000001FF
